:10603700E54670061278958F4622E546B4050612A6
:106047003E3E8F4622E546B40B06126E318F46223E
:10605700E546B40A0612657E8F4622E546B40F066A
:10606700126D9D8F4622E546B41406125FB38F4624
:1060770022E546B419061277D18F4622E546B41EAB
:10608700061278468F4622E546B4230612692F8FFB
:106097004622E546B4280612790D8F4622E546B416
:1060A7002D0612785A8F4622E546B43205127090B3
:0360B7008F4622EF
:1078950090061EE0FFA3E0901CECCFF0A3EFF07F75
:0278A5000522BA
:103E3E0012790950477D047F01125F2B5008E53E31
:103E4E00B401037F0B227D047F02125F2B5008E525
:103E5E003EB402037F0B227D047F03125F2B5008BA
:103E6E00E53EB403037F0B227D047F04125F2B50CB
:103E7E0008E53EB404037F0B227F0A227F081275E9
:103E8E00A550061251887F00227D057F05125F2BFB
:103E9E005023901CEEE07002A3E0701990066CE0C7
:103EAE00FF7C0A7D70126FD5900610E0FFA3E090A4
:103EBE001CEE023F427D067F05125F2B5022901CA6
:103ECE00F0E07002A3E0701890066DE0FF7C0A7DB2
:103EDE0090126FD5900612E0FFA3E0901CF0805474
:103EEE007D077F05125F2B5022901CF2E07002A31B
:103EFE00E0701890066EE0FF7C0A7DB0126FD590D0
:103F0E000614E0FFA3E0901CF280297D087F0512C5
:103F1E005F2B5027901CF4E07002A3E0701D9006FA
:103F2E006FE0FF7C0A7DD0126FD5900616E0FFA3DE
:103F3E00E0901CF4CFF0A3EFF080327D077F0612E5
:103F4E005F2B500F30290C901CECE07002A3E07038
:103F5E0002C22930380C901CECE07002A3E0700213
:103F6E00C238786CE6B405057F041262BA7F05226A
:106E3100203842900633E0901D10F0123202E53EF8
:106E4100B401062049247F0522E53EB40206204D07
:106E5100197F0522E53EB4030620510E7F0522E588
:106E61003EB404062054037F0522901D10E0D39404
:086E71000050C8D2387F0A224C
:10657E00E53B700AE53EB40105753B018028E53B1D
:10658E00700AE53EB40205753B02801AE53B700ABF
:10659E00E53EB40305753B03800CE53B7008E53E14
:1065AE00B40403753B047D077F06125F2B500C7DF0
:1065BE00077F06125F2B501E30291B7D017F0112B3
:1065CE005F2B5012120ECF122A20900650E0FF7C45
:0965DE00067DF0126FD57F0F223B
:106D9D00127909503F120ECF202F092030062031D5
:106DAD0003303209E532700512746B800B786CE696
:106DBD00B4050B7F031262BA122A20120ECF202FB8
:106DCD001020300D20310A203207E5327003122ACF
:0A6DDD00207F0F2212746B7F142236
:105FB300E4F53B900651E0FF7C077D10126FD57D21
:105FC300077F06125F2B500C7D077F06125F2B5055
:105FD30054302951786CE670047F018008786CE6B0
:105FE300B404077F021262BA8038786CE6B40704FF
:105FF3007601802E7D037F05125F2B5025901CF6C2
:10600300E07002A3E0701B900662E0FF7C097D3024
:10601300126FD5900620E0FFA3E0901CF6CFF0A30B
:10602300EFF07F19227D077F06125F2B5005202991
:04603300027F0522C1
:1077D1007D077F06125F2B50062029037F0522902B
:0A77E1000630E0901D10F07F1E221C
:10784600901D10E070037F232212790950037F0AEE
:04785600227F1E224D
:10692F007D047F07125F2B5041E53EB4010B9006AB
:10693F005EE0FF7C087DB0802EE53EB4020B900632
:10694F005FE0FF7C087DD0801EE53EB4030B900610
:10695F0060E0FF7C087DF0800EE53EB4040C9006ED
:10696F0061E0FF7C097D10126FD5900631E0901D1C
:05697F0010F07F28224A
:03790D007F2D22A9
:10785A00901D10E070037F322212790950037F0ACB
:04786A00227F2D222A
:107090003058037F32227D047F05125F2B502890E9
:1070A0001CF8E07002A3E0701E900663E0FF7C090C
:1070B0007D50126FD5900622E0FFA3E0901CF8CF20
:0C70C000F0A3EFF07F3222C2087F002214
:10710500D224753D03123202122A20120ECF1279B3
:10711500095009E53D600512320280F2E4F522F5D9
:10712500231279094009E53D600512320280F2E536
:087135003D70D2C224C25822B1
:04000E0001000041AC
:030003000266AFE3
:0B66AF00C0E0C083C082C0D075D008DE
:1066BA00853082852F83E493FF204404C4540FFF5E
:1066CA00430FF08F80C284D28500C2870000D28730
:1066DA00007580FF7580FEC284C28500C2870000F3
:1066EA000000D287007580FF30440CC2440530E5B3
:0B66FA00307006052F8002D244D2A8A9
:09670500D0D0D082D083D0E03264
:03000B00021A9A3C
:101A9A00C0E0C0F0C083C082C0D075D008758CD8B1
:101AAA00758A92D28C1240981271DCE531D3940077
:101ABA0040051531021E24753114901D10E0D3948F
:101ACA00004003E014F0901D11E0D394004003E0BD
:101ADA0014F0901D12E0D394004003E014F0901D1E
:101AEA0013E0D394004003E014F0E532D3940040AD
:101AFA000215321541E541B40A004003021E219045
:101B0A001B10F8282873021E24021D75021D3D02AF
:101B1A001D10021CA6021C3C021BD2021B68021BDF
:101B2A004B021B2ED3901CEDE09400901CECE09429
:101B3A00005003021E24A3E024FFF0901CEC021EB6
:101B4A0015D3901CE9E09400901CE8E0940050033F
:101B5A00021E24A3E024FFF0901CE8021E157F0158
:101B6A001275334003021E24901CE1E09400901C7D
:101B7A00E0E09400400CA3E024FFF0901CE0E03485
:101B8A00FFF0D3901CEFE09400901CEEE09400402C
:101B9A000CA3E024FFF0901CEEE034FFF0D3901C7D
:101BAA00FBE09400901CFAE094005003021E247D8E
:101BBA00067F01125F2B4003021E24901CFBE024C7
:101BCA00FFF0901CFA021E157F02127533400302C1
:101BDA001E24901CE3E09400901CE2E09400400C68
:101BEA00A3E024FFF0901CE2E034FFF0D3901CF154
:101BFA00E09400901CF0E09400400CA3E024FFF075
:101C0A00901CF0E034FFF0D3901CFDE09400901C8F
:101C1A00FCE094005003021E247D067F02125F2B13
:101C2A004003021E24901CFDE024FFF0901CFC02DD
:101C3A001E157F031275334003021E24901CE5E033
:101C4A009400901CE4E09400400CA3E024FFF09080
:101C5A001CE4E034FFF0D3901CF3E09400901CF2F3
:101C6A00E09400400CA3E024FFF0901CF2E034FF63
:101C7A00F0D3901CFFE09400901CFEE09400500307
:101C8A00021E247D067F03125F2B4003021E24904E
:101C9A001CFFE024FFF0901CFE021E157F04127543
:101CAA00334003021E24901CE7E09400901CE6E0F7
:101CBA009400400CA3E024FFF0901CE6E034FFF00F
:101CCA00D3901CF5E09400901CF4E09400400CA31F
:101CDA00E024FFF0901CF4E034FFF0D3901D01E003
:101CEA009400901D00E094005003021E247D067F9C
:101CFA0004125F2B4003021E24901D01E024FFF012
:101D0A00901D00021E15D3901CEBE09400901CEA73
:101D1A00E09400400CA3E024FFF0901CEAE034FFBA
:101D2A00F0901D14E0D394005003021E24E014F036
:101D3A00021E24D3901CF9E09400901CF8E0940051
:101D4A00400CA3E024FFF0901CF8E034FFF0D3909D
:101D5A001CF7E09400901CF6E094005003021E2445
:101D6A00A3E024FFF0901CF6021E15786CE6FF70C3
:101D7A0003021E24EFB401059006188027786CE64A
:101D8A00FFB40219D3901CEBE09400901CEAE09493
:101D9A0000403FA3E024FFF0901CEA806EEFB403FA
:101DAA001190061AE0FFA3E0901CEACFF0A3EFF02F
:101DBA008020786CE6FFB4041ED3901CEBE09400FC
:101DCA00901CEAE09400400AA3E024FFF0901CEA89
:101DDA008039786C068043EF6405603E786CE6FFD4
:101DEA00B4060D901CEA7402F0A37458F006802A17
:101DFA00EFB40726D3901CEBE09400901CEAE09421
:101E0A0000400EA3E024FFF0901CEAE034FFF080CB
:101E1A0009786C7600800375410A12777E400812B1
:101E2A007339400312779AD0D0D082D083D0F0D0C1
:021E3A00E03294
:03001300025E1377
:0D5E1300C0E0C0F0C083C082C0D075D010C8
:105E200075A0FFC284C285D287C286308018C2A402
:105E3000C2A5D2A6C2A7E5A0540FF54AD2A7FF1269
:105E400063AED286804F308118D2A4C2A5D2A6C23A
:105E5000A7E5A0540FF54AD2A7FF1260BAD28680F8
:105E600034308218C2A4D2A5D2A6C2A7E5A0540F8E
:105E7000F54AD2A7FF12613AD2868019308316D232
:105E8000A4D2A5D2A6C2A7E5A0540FF54AD2A7FF77
:055E90001261BAD28688
:0B5E9500D0D0D082D083D0F0D0E0321B
:1068D800BF0113900632E0901D10F0901D10E0D318
:1068E8009400404280F5BF0213900632E0901D11DB
:1068F800F0901D11E0D39400402C80F5BF03139055
:106908000632E0901D12F0901D12E0D3940040165C
:1069180080F5BF0411900632E0901D13F0901D130E
:07692800E0D3940050F722B8
:10698400304712205D0F900672E0FF7C0B7D3012C1
:106994006FD5D25D22304B12205F0F900673E0FF5B
:1069A4007C0B7D50126FD5D25F22304E1220600FC7
:1069B400900674E0FF7C0B7D70126FD5D26022309C
:1069C400521120610E900675E0FF7C0B7D90126FD2
:0469D400D5D2612295
:10540800303D1A204617900664E0FF7C097D701233
:105418006FD5D246C214C210C21CC218223046141C
:10542800203911900665E0FF7C097D90126FD5C286
:1054380046C23D22303E1A204817900666E0FF7C9F
:10544800097DB0126FD5D248C215C211C21DC2194A
:1054580022304814203A11900667E0FF7C097DD07D
:10546800126FD5C248C23E2230401A204C1790060F
:1054780068E0FF7C097DF0126FD5D24CC216C212CB
:10548800C21EC21A22304C14203B11900669E0FF5C
:105498007C0A7D10126FD5C24CC2402230421A20BD
:1054A8004F1790066AE0FF7C0A7D30126FD5D24F05
:1054B800C217C213C21FC21B22304F13203C1090C8
:1054C800066BE0FF7C0A7D50126FD5C24FC24222A4
:104FD100123F7ED28C7F071275A5500512001680F4
:104FE10012126EC17F1F7E0012755A90001FEFF0E2
:104FF1001273937F081275A5500512570D80FE900C
:1050010006087402F0A37458F090060A7402F0A323
:105011007458F090060C7402F0A37458F090060EC8
:105021007402F0A37458F0900681E0FF7C0D7D10AE
:10503100126FD5E4FFEFFD3395E0FC74302DF5825E
:1050410074003CF583E0FE74F02DF582741A3CF592
:1050510083EEF00FBF08DED20812779A7545017F03
:10506100011262BA900618E0FFA3E0901CEACFF0AB
:10507100A3EFF0C20812779A123202126037305948
:1050810003124CF4305A031244E1305B031245EB36
:10509100305E031246F5124B047D077F06125F2B2B
:0C50A1004002C22912540812698480CC1D
:104CF4007C007D80C2657F0112357150077F0112EF
:104D04001E3C80707C007D70D2657F01123571502D
:104D140002800D7C007D78D2657F011235715007C9
:104D24007F0112085D804D7C007DA0D2657F011259
:104D3400357150117D077F06125F2B5008754501B0
:104D4400127494802F7C007DA8C2657F0112357196
:104D540050107D057F01125F2B50077F011241B077
:104D640080127C007DB0C2657F0112357150057FD1
:104D740001124DEAE4F54CAF4CEF3395E0FEEF78C9
:104D840003C333CE33CED8F92400F58274013EAD8B
:104D940082FCD2657F011235715038754501AF4CE4
:104DA400EF3395E0FE74A02FF58274063EF583E0A0
:104DB400FFC007AF4CEF3395E0FEEF7805C333CE69
:104DC40033CED8F924F0F58274103EAD82FCD007BE
:104DD400126BCD054CC3E54C648094A84099C2592C
:054DE400C2631269D852
:014DE90022A7
:1044E1007D017F06125F2B503D7C007D88C2657F78
:1044F10002123571500BD2097F02121E3CC2098093
:10450100257C007D70D2657F021235715002800DCD
:104511007C007D78D2657F021235715009D2097F06
:104521000212085DC20990001FE030E1427C007D6B
:10453100A0D2657F0212357150147D077F06125F8C
:104541002B500B127580754502127494801E7C00ED
:104551007DA8C2657F0212357150147D057F02125C
:104561005F2B500B1275807F021241B01276757D60
:10457100027F06125F2B506AE4F54CAF4CEF339586
:10458100E0FEEF7803C333CE33CED8F92400F582B1
:1045910074013EAD82FCD2657F02123571503875CF
:1045A1004502AF4CEF3395E0FE74A02FF5827406FF
:1045B1003EF583E0FFC007AF4CEF3395E0FEEF78A7
:1045C10005C333CE33CED8F924F0F58274103EAD55
:1045D10082FCD007126BCD054CC3E54C648094A8D6
:0945E1004099C25AC264126A2C0E
:0145EA0022AE
:1045EB007D037F06125F2B503D7C007D90C2657F63
:1045FB0003123571500BD20E7F03121E3CC20E807C
:10460B00257C007D70D2657F031235715002800DC1
:10461B007C007D78D2657F031235715009D20E7FF5
:10462B000312085DC20E90001FE030E2427C007D59
:10463B00A0D2657F0312357150147D077F06125F80
:10464B002B500B127580754503127494801E7C00E1
:10465B007DA8C2657F0312357150147D057F03124F
:10466B005F2B500B1275807F031241B01276757D54
:10467B00047F06125F2B506AE4F54CAF4CEF339579
:10468B00E0FEEF7803C333CE33CED8F92400F582A6
:10469B0074013EAD82FCD2657F03123571503875C3
:1046AB004503AF4CEF3395E0FE74A02FF5827406F3
:1046BB003EF583E0FFC007AF4CEF3395E0FEEF789C
:1046CB0005C333CE33CED8F924F0F58274103EAD4A
:1046DB0082FCD007126BCD054CC3E54C648094A8CB
:0946EB004099C25BC228126A80EA
:0146F40022A3
:1046F5007D057F06125F2B503D7C007D98C2657F4E
:1047050004123571500BD20C7F04121E3CC20C8072
:10471500257C007D70D2657F041235715002800DB5
:104725007C007D78D2657F041235715009D20C7FEB
:104735000412085DC20C90001FE030E3427C007D4E
:10474500A0D2657F0412357150147D077F06125F74
:104755002B500B127580754504127494801E7C00D5
:104765007DA8C2657F0412357150147D057F041242
:104775005F2B500B1275807F041241B01276757D48
:10478500067F06125F2B506AE4F54CAF4CEF33956C
:10479500E0FEEF7803C333CE33CED8F92400F5829B
:1047A50074013EAD82FCD2657F04123571503875B7
:1047B5004504AF4CEF3395E0FE74A02FF5827406E7
:1047C5003EF583E0FFC007AF4CEF3395E0FEEF7891
:1047D50005C333CE33CED8F924F0F58274103EAD3F
:1047E50082FCD007126BCD054CC3E54C648094A8C0
:0947F5004099C25EC22A126AD486
:0147FE002298
:106C6D00BF010AC214C210C21CC2188025BF020A7D
:106C7D00C215C211C21DC2198018BF030AC216C2A5
:106C8D0012C21EC21A800BBF0408C217C213C21F44
:106C9D00C21B90001FE0FF30E002D224EF30E10272
:0E6CAD00D225EF30E202D226EF30E302D227EA
:016CBB0022B6
:1063AE008F4B7868E6C39450506E30496B7D077FF3
:1063BE0001125F2B502B205C287868E6700D90063A
:1063CE003BE0B54B06203F03D23F22202F0D203F4E
:1063DE000A7F01126C6D753D02D22F900634E0F5E6
:1063EE00327D087F06125F2B501990063FE0B54BA9
:1063FE0006205C03D263220534E534AE33700E05FD
:10640E0033800A0534E534AE337002053314F58259
:09641E008E83E54BF0786806223C
:1060BA008F4B7869E6C394505075304D727D077FD7
:1060CA0002125F2B50327F02127533502B205C284C
:1060DA007869E6700D90063BE0B54B06204103D285
:1060EA00412220300D20410A7F02126C6D753D025B
:1060FA00D230900634E0F5327D087F06125F2B50CD
:10610A001990063FE0B54B06205C03D2642205369F
:10611A00E536AE35700E0535800A0536E536AE35FC
:10612A007002053514F5828E83E54BF078690622F4
:10613A008F4B786AE6C3945050753051727D077F51
:10614A0003125F2B50327F03127533502B205C28C9
:10615A00786AE6700D90063BE0B54B06204303D201
:10616A00432220310D20430A7F03126C6D753D02D4
:10617A00D231900634E0F5327D087F06125F2B504B
:10618A001990063FE0B54B06205C03D22822053859
:10619A00E538AE37700E0537800A0538E538AE3770
:1061AA007002053714F5828E83E54BF0786A062271
:1061BA008F4B786BE6C3945050753054727D077FCD
:1061CA0004125F2B50327F04127533502B205C2847
:1061DA00786BE6700D90063BE0B54B06204503D27E
:1061EA00452220320D20450A7F04126C6D753D024E
:1061FA00D232900634E0F5327D087F06125F2B50CA
:10620A001990063FE0B54B06205C03D22A22053AD4
:10621A00E53AAE39700E0539800A053AE53AAE39E3
:10622A007002053914F5828E83E54BF0786B0622ED
:1075800090001FE0FF30E004D208D220EF30E10489
:10759000D209D221EF30E204D20ED222EF30E3043E
:0575A000D20CD22322F1
:10767500C220C221C222C22390001FE0FF30E102D6
:0F768500C209EF30E202C20EEF30E302C20C2264
:1062BA008F4CE54CB401197D017F05125F2B500C00
:1062CA0090065AE0FF7C087D30126FD5786C062262
:1062DA00E54CB402177D027F05125F2B50479006EA
:1062EA005BE0FF7C087D50126FD58039E54CB40421
:1062FA001A7D027F05125F2B500C90065DE0FF7C31
:10630A00087D90126FD5786C760622E54CB4031995
:10631A007D027F05125F2B500C90065CE0FF7C0823
:0A632A007D70126FD5786C760122A9
:1077B600EF1FAA0670011ED39400EA9400400BE462
:0A77C600FDEDC394C850E90D80F7F3
:0177D0002296
:1057C2008F5D30695BE55DB40111D22090001FE06E
:1057D200F420E003305C44D2088040E55DB402115D
:1057E200D22190001FE0F420E103305C2ED2098028
:1057F2002AE55DB40311D22290001FE0F420E203F7
:10580200305C18D20E8014E55DB4040FD2239000F0
:105812001FE0F420E303305C02D20CAF5D0268D8D3
:10582200E55DB40110C22090001FE0F420E00330D7
:105832005C41C20822E55DB40210C22190001FE063
:10584200F420E103305C2CC20922E55DB40310C2EE
:105852002290001FE0F420E203305C17C20E22E522
:105862005DB4040FC22390001FE0F420E303305C18
:0458720002C20C2240
:105876008F5230675BE552B40111D22490001FE0CD
:10588600F420E003305C44D2088040E552B40211B3
:10589600D22590001FE0F420E103305C2ED209806F
:1058A6002AE552B40311D22690001FE0F420E20349
:1058B600305C18D20E8014E552B4040FD227900043
:1058C6001FE0F420E303305C02D20CAF520268D82A
:1058D600E552B40110C22490001FE0F420E003302A
:1058E6005C41C20822E552B40210C22590001FE0B6
:1058F600F420E103305C2CC20922E552B40310C245
:105906002690001FE0F420E203305C17C20E22E569
:1059160052B4040FC22790001FE0F420E303305C6A
:0459260002C20C228B
:0827CA008F538C548D558B5682
:1027D200C265E55524FFF582E55434FFF583E0F543
:1027E20058855582855483E0FFF559A3E0FEF55ADA
:1027F200EF14B40800505C90280775F003A4C58359
:1028020025F0C5837302281F02282602282D0228DC
:102812003402283B022842022849022850755701F7
:10282200D265802F755702D2658028755704D2650C
:102832008021755708D265801A755710D2658013AA
:10284200755720D265800C755740D2658005755743
:1028520080D265EE24FE700302291724F8605C24FE
:10286200096003022929E553B4010590002080453F
:10287200E553B40205900021803BE553B403059073
:1028820000228031E553B404059000238027E553EC
:10289200B40505900024801DE553B406059000257B
:1028A2008013E553B407059000268009E5536408B8
:1028B2007077900027E04557F0806EE553B401052C
:1028C2009000208045E553B40205900021803BE54D
:1028D20053B403059000228031E553B404059000FF
:1028E200238027E553B40505900024801DE553B4E9
:1028F20006059000258013E553B407059000268055
:1029020009E55364087022900027E0FFE557F4FEC2
:10291200EF5EF08014E553B4080D8555828554832B
:10292200E0FF125D7FC265C265206503022A1FE5D2
:1029320053B40109900020E0FD7F208060E553B48C
:102942000209900021E0FD7F218052E553B4030982
:10295200900022E0FD7F228044E553B404099000F8
:1029620023E0FD7F238036E553B40509900024E07F
:10297200FD7F248028E553B40609900025E0FD7F01
:1029820025801AE553B40709900026E0FD7F2680D2
:102992000CE553B4080C900027E0FD7F277E00125F
:1029A2007015D2AFD269AF561257C2AD58E4FF12BA
:1029B2007417AD59E4FF127417E55AB401047D3857
:1029C2008007E55AB40A077D367F06127417E5536D
:1029D200B408031273937D077F06125F2B500B20FE
:1029E2002908C208C209C20EC20C7D017F01125F12
:1029F2002B4002C2087D017F02125F2B4002C209F6
:102A02007D017F03125F2B4002C20E7D017F041203
:0D2A12005F2B4002C20CC269AF561257C2C2
:012A1F002294
:045B18008F538D54C6
:105B1C00D269AF541257C2AF541268D8E553B401CE
:105B2C00059000208044E553B40205900021803A92
:105B3C00E553B403059000228030E553B40405907E
:105B4C0000238026E553B40505900024801CE55302
:105B5C00B406059000258012E553B4070590002685
:105B6C008008E553B40806900027E0F555E555602C
:105B7C0025755701E4F556E55530E007AD57E4FFC0
:105B8C00127417E555C313F55505570556E556C35D
:105B9C00940840E3800E7D187F021274177D537FAA
:0B5BAC0002127417C269AF541257C2F6
:015BB70022CB
:021E3C008F4DC8
:101E3E00E54D6401701E754E1B754F10900080E0CD
:101E4E00F550E54F2550F582E4354EF583E0F55219
:101E5E0078688069E54D6402701E754E1B754F6083
:101E6E00900088E0F550E54F2550F582E4354EF5AB
:101E7E0083E0F55278698045E54D6403701E754E1A
:101E8E001B754FB0900090E0F550E54F2550F58250
:101E9E00E4354EF583E0F552786A8021E54DB404C1
:101EAE001F754E1C754F00900098E0F550E54F25BC
:101EBE0050F582E4354EF583E0F552786BE6F55138
:101ECE00E55214B4090040030221DB901EE775F0C1
:101EDE0003A4C58325F0C58373021F02021F55029A
:101EEE001FA8021FFB02204E0220A10220F4022195
:101EFE0045022195E54F2550F582E4354EF583A335
:101F0E00E0B40A18E5502402FFE433FEE551B507AC
:101F1E000BE4B50607AD4D7F0102216AAF507E007E
:101F2E00EF2403FDEE33FCE5516D7001EC6003020E
:101F3E0021DBEF254FFFEE354ECF2401FDE43FFCB4
:101F4E00AB4D7F01022192E54F2550F582E4354ECF
:101F5E00F583A3E0B40A18E5502402FFE433FEE54E
:101F6E0051B5070BE4B50607AD4D7F0202216AAFEE
:101F7E00507E00EF2403FDEE33FCE5516D7001EC55
:101F8E0060030221DBEF254FFFEE354ECF2401FD1E
:101F9E00E43FFCAB4D7F02022192E54F2550F582C6
:101FAE00E4354EF583A3E0B40A18E5502402FFE4AD
:101FBE0033FEE551B5070BE4B50607AD4D7F0302C1
:101FCE00216AAF507E00EF2403FDEE33FCE5516D28
:101FDE007001EC60030221DBEF254FFFEE354ECF93
:101FEE002401FDE43FFCAB4D7F03022192E54F251A
:101FFE0050F582E4354EF583A3E0B40A18E550247B
:10200E0002FFE433FEE551B5070BE4B50607AD4D0F
:10201E007F0402216AAF507E00EF2403FDEE33FCF5
:10202E00E5516D7001EC60030221DBEF254FFFEEF1
:10203E00354ECF2401FDE43FFCAB4D7F04022192CF
:10204E00E54F2550F582E4354EF583A3E0B40A182A
:10205E00E5502402FFE433FEE551B5070BE4B50667
:10206E0007AD4D7F0502216AAF507E00EF2403FDC0
:10207E00EE33FCE5516D7001EC60030221DBEF25C0
:10208E004FFFEE354ECF2401FDE43FFCAB4D7F05F7
:10209E00022192E54F2550F582E4354EF583A3E0FB
:1020AE00B40A18E5502402FFE433FEE551B5070BE0
:1020BE00E4B50607AD4D7F0602216AAF507E00EFF4
:1020CE002403FDEE33FCE5516D7001EC600302213B
:1020DE00DBEF254FFFEE354ECF2401FDE43FFCAB89
:1020EE004D7F06022192E54F2550F582E4354EF5DF
:1020FE0083A3E0B40A17E5502402FFE433FEE55152
:10210E00B5070AE4B50606AD4D7F07804FAF507E8A
:10211E0000EF2403FDEE33FCE5516D7001EC60031E
:10212E000221DBEF254FFFEE354ECF2401FDE43FBC
:10213E00FCAB4D7F07804DE54F2550F582E4354EC3
:10214E00F583A3E0B40A18E5502402FFE433FEE55C
:10215E0051B5070BE4B50607AD4D7F08025B18AF0E
:10216E00507E00EF2403FDEE33FCE5516D7001EC63
:10217E00705BEF254FFFEE354ECF2401FDE43FFCA3
:10218E00AB4D7F080227CAE54F2550F582E4354E48
:10219E00F583A3A3E07036E54F2550F582E4354E66
:1021AE00F583A3E024F96008147022AF4D02750C7C
:1021BE00D2697F011257C2AF4D1268D87D5E7F0281
:0D21CE00127417C2697F011257C212570D1B
:0121DB0022E1
:043571008C4D8D4EA2
:10357500054EE54E7002054D14F5828C83E0F97019
:1035850003023713BF010875331B753410801FBF45
:10359500020875351B7536608014BF030875371B27
:1035A5007538B08009BF040675391C753A00206569
:1035B50003023679BF01087868E6696002C322BF55
:1035C50002087869E6696002C322BF0308786AE6E3
:1035D500696002C322BF0408786BE6696002C322F2
:1035E500E4FEEEC3994003023677EF6401701CE5F3
:1035F5004E2EF582E4354DF583E0FDE5342EF5825A
:10360500E43533F583E06D6002C322EF6402701C7C
:10361500E54E2EF582E4354DF583E0FDE5362EF5D4
:1036250082E43535F583E06D6002C322EF640370F3
:103635001CE54E2EF582E4354DF583E0FDE5382E8B
:10364500F582E43537F583E06D6002C322EF64044B
:10365500701CE54E2EF582E4354DF583E0FDE53A27
:103665002EF582E43539F583E06D6002C3220E0242
:1036750035E7D322306503023714E4FEEEC39940E3
:1036850003023711EF6401701CE54E2EF582E43517
:103695004DF583E0FDE5342EF582E43533F583E021
:1036A5006D6065C322EF6402701CE54E2EF582E461
:1036B500354DF583E0FDE5362EF582E43535F583A8
:1036C500E06D6044C322EF6403701CE54E2EF58265
:1036D500E4354DF583E0FDE5382EF582E43537F523
:1036E50083E06D6023C322EF6404701CE54E2EF564
:1036F50082E4354DF583E0FDE53A2EF582E4353972
:0F370500F583E06D6002C3220E023681D322C32A
:013714002292
:102A200090001FE0540FF55CB4010BE53EB40103C8
:102A3000D21422C21422E55C6403702AE53EB4017C
:102A400006D214D2108004C214C210E53EB40211A2
:102A5000D2157D017F07125F2B4003022C3BD21160
:102A600022C215C21122E55C6405702AE53EB4015C
:102A700006D214D21C8004C214C21CE53EB4031159
:102A8000D2167D027F07125F2B4003022C3BD21E21
:102A900022C216C21E22E55C6409702AE53EB4011A
:102AA00006D214D2188004C214C218E53EB4041130
:102AB000D2177D037F07125F2B4003022C3BD21BF2
:102AC00022C217C21B22E55C6407704EE53EB401CA
:102AD00008D214D210D21C8006C214C210C21CE547
:102AE0003EB40211D2157D017F07125F2B5002D236
:102AF00011D21D8006C215C211C21DE53EB40313DA
:102B0000D216D2127D027F07125F2B4003022C3BAC
:102B1000D21E22C216C212C21E22E55C640B704E87
:102B2000E53EB40108D214D210D2188006C214C2F5
:102B300010C218E53EB40211D2157D017F07125F65
:102B40002B5002D211D2198006C215C211C219E54A
:102B50003EB40413D217D2137D037F07125F2B40BC
:102B600003022C3BD21B22C217C213C21B22E55CFC
:102B7000640D704BE53EB40108D214D21CD218800B
:102B800006C214C21CC218E53EB40311D2167D025F
:102B90007F07125F2B5002D21ED21A8006C216C2C5
:102BA0001EC21AE53EB40413D217D21F7D037F075D
:102BB000125F2B4003022C3BD21B22C2178078E508
:102BC0005C640F7076E53EB4010AD214D210D21CB8
:102BD000D2188008C214C210C21CC218E53EB4024A
:102BE00013D2157D017F07125F2B5002D211D21D27
:102BF000D2198008C215C211C21DC219E53EB40324
:102C000013D216D2127D027F07125F2B5002D21E02
:102C1000D21A8008C216C212C21EC21AE53EB404FD
:102C200012D217D213D21F7D037F07125F2B500BD6
:0B2C3000D21B22C217C213C21FC21B1E
:012C3B002276
:100ECF0090001FE0540FF55CB4010F7D017F0112FC
:100EDF005F2B5003D20822C20822E55C64037054D2
:100EEF00E53E6401701E7D017F01125F2B5004D21D
:100EFF00088002C2087D017F02125F2B5003D209C6
:100F0F0022C20922E53E640260030213477D017F7E
:100F1F0001125F2B5004D2088002C2087D017F02AC
:100F2F00125F2B500C7D017F07125F2B5003D209EC
:100F3F0022C20922E55C64057054E53E6401701E0F
:100F4F007D017F01125F2B5004D2088002C2087D01
:100F5F00017F03125F2B5003D20E22C20E22E53EF9
:100F6F00640360030213477D017F01125F2B50045E
:100F7F00D2088002C2087D017F03125F2B500C7DC7
:100F8F00027F07125F2B5003D20E22C20E22E55CA6
:100F9F0064097054E53E6401701E7D017F01125F8C
:100FAF002B5004D2088002C2087D017F04125F2BF0
:100FBF005003D20C22C20C22E53E640460030213DC
:100FCF00477D017F01125F2B5004D2088002C208B7
:100FDF007D017F04125F2B500C7D037F07125F2B67
:100FEF005003D20C22C20C22E55C6407600302108E
:100FFF00AEE53E6401702D7D017F01125F2B500421
:10100F00D2088002C2087D017F02125F2B5004D2EA
:10101F00098002C2097D017F03125F2B5003D20E9C
:10102F0022C20E22E53E640270367D017F01125FFF
:10103F002B5004D2088002C2087D017F02125F2B61
:10104F00500D7D017F07125F2B5004D2098002C221
:10105F00097D017F03125F2B5003D20E22C20E2295
:10106F00E53E640360030213477D017F01125F2B8E
:10107F005004D2088002C2087D017F02125F2B50FC
:10108F0004D2098002C2097D017F03125F2B500C2D
:10109F007D027F07125F2B5003D20E22C20E22E574
:1010AF005C640B6003021165E53E6401702D7D01E8
:1010BF007F01125F2B5004D2088002C2087D017F8E
:1010CF0002125F2B5004D2098002C2097D017F04F6
:1010DF00125F2B5003D20C22C20C22E53E64027029
:1010EF00367D017F01125F2B5004D2088002C208A7
:1010FF007D017F02125F2B500D7D017F07125F2B49
:10110F005004D2098002C2097D017F04125F2B5067
:10111F0003D20C22C20C22E53E6404600302134783
:10112F007D017F01125F2B5004D2088002C2087D1F
:10113F00017F02125F2B5004D2098002C2097D0188
:10114F007F04125F2B500C7D037F07125F2B500320
:10115F00D20C22C20C22E55C640D600302121CE566
:10116F003E6401702D7D017F01125F2B5004D20868
:10117F008002C2087D017F03125F2B5004D20E80C4
:10118F0002C20E7D017F04125F2B5003D20C22C2CC
:10119F000C22E53E640370367D017F01125F2B50F8
:1011AF0004D2088002C2087D017F03125F2B500D0D
:1011BF007D027F07125F2B5004D20E8002C20E7D7C
:1011CF00017F04125F2B5003D20C22C20C22E53E8A
:1011DF00640460030213477D017F01125F2B5004EB
:1011EF00D2088002C2087D017F03125F2B5004D208
:1011FF000E8002C20E7D017F04125F2B500C7D0307
:10120F007F07125F2B5003D20C22C20C22E55C64C5
:10121F000F6003021347E53E6401703C7D017F01BF
:10122F00125F2B5004D2088002C2087D017F021288
:10123F005F2B5004D2098002C2097D017F03125F28
:10124F002B5004D20E8002C20E7D017F04125F2B41
:10125F005003D20C22C20C22E53E640270457D0180
:10126F007F01125F2B5004D2088002C2087D017FDC
:10127F0002125F2B500D7D017F07125F2B5004D29E
:10128F00098002C2097D017F03125F2B5004D20E29
:10129F008002C20E7D017F04125F2B5003D20C22FD
:1012AF00C20C22E53E640370457D017F01125F2B66
:1012BF005004D2088002C2087D017F02125F2B50BA
:1012CF0004D2098002C2097D017F03125F2B500DEA
:1012DF007D027F07125F2B5004D20E8002C20E7D5B
:1012EF00017F04125F2B5003D20C22C20C22E53E69
:1012FF00640470447D017F01125F2B5004D208807B
:10130F0002C2087D017F02125F2B5004D2098002B6
:10131F00C2097D017F03125F2B5004D20E8002C2DF
:10132F000E7D017F04125F2B500C7D037F07125F30
:08133F002B5003D20C22C20C5A
:011347002283
:1076D0007F01127533500CE53BB40107C209C20E9D
:0D76E000C20C227F011275334002C2082245
:1076ED007F02127533500CE53BB40207C209C20E7E
:0D76FD00C20C227F021275334002C2092226
:10770A007F03127533500CE53BB40307C209C20E5E
:0D771A00C20C227F031275334002C20E2202
:107727007F04127533500CE53BB40407C209C20E3F
:0D773700C20C227F041275334002C20C22E6
:10670E000500050105030507050F051F051E051CE0
:10671E00051805100201040E040A03060101040BFC
:10672E000304040F020304010302040D020002021B
:10673E00030004090404030503070100030304070F
:10674E00030104060402040C0516051500000615C7
:0E675E00062A060C06380633061E061206171B
:1050AD00203737900640E004F519D3648094815081
:1050BD0003025187D3E5196480948F400375190F4E
:1050CD0090063DE0FF123B9F90063EE0F518E4F59B
:1050DD001ED237C262C257C24A22304A60306216AF
:1050ED00152EE52ED394004003025187C2CAC26229
:1050FD00D25785182E2230570E152EE52ED394003B
:10510D005078C262C25722AF1C151CEF700BC24AF9
:10511D00E51825E0F52ED25722E51D30E00585185E
:10512D002E8008E51875F003A4F52EAF1D7801EF5C
:10513D0008800103D8FDF51DD262D2CA22D5190807
:10514D00C237E4F53DC25822051E7440251EF58276
:10515D00E43406F583E025E0240EF582E43467F5AA
:10516D0083E493540FF51C740193F51D700AD25707
:0A517D00E51825E025E0F52ED24AE2
:015187002205
:105C510020371A90063DE0FF123B9F90063EE0F58B
:105C61001AE4F51ED237C262C257C24A22304A59DB
:105C7100306213152EE52ED39400506BC2CAC26256
:105C8100D257851A2E2230570E152EE52ED39400A9
:105C91005055C262C25722AF1C151CEF7007C24A91
:105CA100C237F53D22E51D30E005851A2E8008E555
:105CB1001A75F003A4F52EAF1D7801EF08800103DA
:105CC100D8FDF51DD262D2CA22E53F25E0240EF5AA
:105CD10082E43467F583E493FA740193FBEA540F89
:075CE100F51CEBF51DD24A92
:015CE8002299
:10786E00C3EF648094A15008EF25E025E0F52E22A9
:04787E00E4F52E22DD
:1071A800BF010790063E7418F022BF020790063E02
:1071B8007412F022BF030590063E8014BF040790A6
:1071C800063E740BF02290063EBF05047409F022B7
:0471D800740CF02221
:103B9F00EF14B420004003023CF2903BB775F003E2
:103BAF00A4C58325F0C58373023C17023C1E023C5B
:103BBF0025023C2C023C33023C3A023C41023C4879
:103BCF00023C4F023C56023C5D023C64023C6B02DD
:103BDF003C72023C79023C80023C87023C8E023CE4
:103BEF0095023C9C023CA3023CAA023CB1023CB8A9
:103BFF00023CBF023CC6023CCD023CD4023CD60282
:103C0F003CDD023CE4023CEB75CB8E75CAC62275D7
:103C1F00CB9575CA772275CB9B75CA692275CBA0D8
:103C2F0075CABA2275CBA675CA332275CBAB75CAC6
:103C3F00632275CBB075CA022275CBB475CAA322A5
:103C4F0075CBB875CAFA2275CBBC75CAD82275CB9D
:103C5F00C075CAA82275CBC475CA362275CBC77575
:103C6F00CA862275CBCA75CABC2275CBCD75CAB4AC
:103C7F002275CBD075CA762275CBD375CA30227513
:103C8F00CBD575CAB22275CBD875CA132275CBDACC
:103C9F0075CA522275CBDC75CA7D2275CBDD75CA0C
:103CAF006E2275CBE075CA542275CBE275CA1B2202
:103CBF0075CBE375CAC32275CBE575CA5E2275CB8A
:103CCF00E675CADA22801C75CBE875CA902275CBCF
:103CDF00EA75CAD92275CBEC75CA092275CBED7579
:0A3CEF00CA292275CBE875CA4122EC
:106F0900EFC39400403FEF9408503AE4FEEF75F068
:106F190008A42428F582E43400F583E5822EF5825D
:106F2900E43583F583E0FCED75F008A424E8F582E7
:106F3900E4341AF583E5822EF582E43583F583EC92
:056F4900F00EBE08C8B7
:016F4E002220
:105D7F008F5BE55B6405701D200A0DD20A7FF47EF0
:105D8F00011277B6C20A8074C20A7FF47E011277BD
:105D9F00B6D20A8067E55B6406701D200B0DD20B2F
:105DAF007FF47E011277B6C20B800BC20B7FF47E9D
:105DBF00011277B6D20B8044E55B6407701D200F8C
:105DCF000DD20F7FF47E011277B6C20F800BC20F78
:105DDF007FF47E011277B6D20F8021E55B640870E5
:105DEF0022200D0DD20D7FF47E011277B6C20D80E9
:105DFF000BC20D7FF47E011277B6D20D7FF47E01B8
:045E0F001277B6222E
:104B0400A233B330B401B350357D017F08125F2B5B
:104B14005027A233B35010A2B4B3500B900652E006
:104B2400FF7C077D30800F30330F30B40C90065378
:104B3400E0FF7C077D50126FD5A2B4B39233A23448
:104B4400B330B501B350357D027F08125F2B502777
:104B5400A234B35010A2B5B3500B900654E0FF7CBE
:104B6400077D70800F30340F30B50C900655E0FF90
:104B74007C077D90126FD5A2B5B39234A235B330C1
:104B8400B701B350357D037F08125F2B5027A23540
:104B9400B35010A2B7B3500B900656E0FF7C077DCC
:104BA400B0800F30350F30B70C900657E0FF7C070C
:104BB4007DD0126FD5A2B7B39235A236B330B60109
:104BC400B350357D047F08125F2B5027A236B350B3
:104BD40010A2B6B3500B900658E0FF7C077DF0801E
:104BE4000F30360F30B60C900659E0FF7C087D106C
:094BF400126FD5A2B6B39236226D
:10739300900027E0FF30E404D20A8002C20AEF30F3
:1073A300E504D20B8002C20BEF30E604D20F800259
:0B73B300C20FEF30E703D20D22C20D25
:0173BE0022AC
:10713D0090063CE0FF602E20370F6029123B9FD256
:10714D00CAD237D262752E1422E52ED39400400395
:10715D00152E22206208D2CA752E14D26222C2CAFE
:06716D00752E7DC26222B6
:107173002037127F1C123B9FD2CAD237D262752EA0
:1071830064751B3C22E52ED394004003152E22AFD9
:107193001B151BD3EF648094804004752E6422C2B8
:0471A30037E4F53D9B
:0171A70022C5
:104BFD0020371C754006E53E75F008A424E8F582C3
:104C0D00E4341AF583E06003D23722E4F53D22E562
:104C1D002ED394004003152E22C2CA1540E5401430
:104C2D007003024CB814606F14604014602E146051
:104C3D0003024CECE53E75F008A424E8F582E4345B
:104C4D001AF583E0FF7003F53D22123B9FE53E759B
:104C5D00F008A424E9F582E4341A8079E53E75F074
:104C6D0008A424EAF582E4341A80397408441B70D0
:104C7D0003F53D22E53E75F008A424EBF582E434FE
:104C8D001AF583E0FF123B9FE53E75F008A424EC76
:104C9D00F582E4341A803EE53E75F008A424EDF566
:104CAD0082E4341AF583E0FF02786E7420441B70A1
:104CBD0003F53D22E53E75F008A424EEF582E434BB
:104CCD001AF583E0FF123B9FE53E75F008A424EF33
:104CDD00F582E4341AF583E0FF12786ED2CA22E42D
:074CED00F53DC2CAC23722E7
:1071DC00E53D14601C14601C14601C14601F1460CA
:1071EC001F2405701EC2CAC237C262C257E4F540E2
:1071FC0022024BFD02713D1250ADD2582202717326
:04720C00125C51229D
:10733900E52365437004E5226542601F8522428585
:107349002343C2A4D2A5C2A6C2A700AF2312781BA9
:0D735900E522FF12781B00D2A7D322C32229
:10777E00E52465446014852444D2A4D2A5C2A6C2D1
:0C778E00A7AF2412781BD2A7D322C3227D
:10779A00E521653C601485213CD2A4C2A5C2A6C2DB
:0C77AA00A7AF2112781BD2A7D322C32264
:103F7E00E4F54CF54D754E1E754FFF854D82854C03
:103F8E0083E0F5506350FFE550F0E065506003129A
:103F9E0079106350FF854D82854C83E550F0E065C6
:103FAE00506003127910054DE54D7002054CE54F3A
:103FBE00154F7002154ED3E54F9400E54E94005008
:103FCE00BAE4F54CF54DF54EF54FE54D254FF5821E
:103FDE00E54C354EF583E4F0054FE54F7002054E86
:103FEE00B4FFE7E54EB41EE275985A7589217588BF
:103FFE0045758845758DE775878075C90275331BC4
:10400E0075341075351B75366075371B7538B07580
:10401E00391C753A0075B701D2A9D2A8D2AA90065A
:10402E0000E0FFA3E0901CE0CFF0A3EFF0900602BB
:10403E00E0FFA3E0901CE2CFF0A3EFF0900604E0C7
:10404E00FFA3E0901CE4CFF0A3EFF0900606E0FF94
:10405E00A3E0901CE6CFF0A3EFF0901CFA7417F0DB
:10406E00A37499F0901CFC7417F0A37499F0901C33
:10407E00FE7417F0A37499F0901D007417F0A374DA
:09408E0099F0D291D2AF127441F5
:014097002206
:0279100080FEF7
:1075A500C2AFC284D285BF070AC286E580A2E29235
:1075B50066800BBF0808C286E580A2E39266D28684
:0475C500D2AFA26639
:0175C900229F
:105F2B00BF0107900020E0FE8048BF0207900021D0
:105F3B00E0FE803EBF0307900022E0FE8034BF04EA
:105F4B0007900023E0FE802ABF0507900024E0FEA7
:105F5B008020BF0607900025E0FE8016BF07079044
:105F6B000026E0FE800CBF0807900027E0FE8002B1
:105F7B00E4FEBD0103EE1322BD0204EEA2E122BD3D
:105F8B000304EEA2E222BD0404EEA2E322BD05044B
:105F9B00EEA2E422BD0604EEA2E522BD0704EEA2AA
:075FAB00E622BD0802EE33FF
:015FB20022CC
:024DEA008F4DEB
:104DEC009000B0E0F54EE54D64017037E54E2402BD
:104DFC00FFE433FE7868E66F7001EE6003024EDF6D
:104E0C007410254EF582E4341BAF82F5508F51D2CD
:104E1C00697F011257C2127744123715C2697F019C
:104E2C00024EDCE54D64027037E54E2402FFE4339C
:104E3C00FE7869E66F7001EE6003024EDF74602548
:104E4C004EF582E4341BAF82F5508F51D2697F024C
:104E5C001257C2127744123715C2697F02024EDC18
:104E6C00E54D64037033E54E2402FFE433FE786AAB
:104E7C00E66F7001EE705C74B0254EF582E4341B65
:104E8C00AF82F5508F51D2697F031257C21277440B
:104E9C00123715C2697F038037E54D64047034E521
:104EAC004E2402FFE433FE786BE66F7001EE702344
:104EBC007400254EF582E4341CAF82F5508F51D22C
:104ECC00697F041257C2127744123715C2697F04E6
:034EDC001257C2A8
:014EDF0022B0
:043715008F4FE4FDF1
:023719008D57CA
:10371B0075F020EFA42460F582E5F03403AF82F559
:10372B005A8F5BF583E0F558D3940050030238A110
:10373B00E558941040030238A1E557704C7FF47E96
:10374B00011277B6E55825E0F558755901E558246F
:10375B0001FFE433FEC3E5599FEE6480F874809853
:10376B0040030238A1E55B2559F582E4355AF58310
:10377B00E0FFE55B2559F582E4355AF583A3E0FDBF
:10378B001274170559055980C4E5576401707AC244
:10379B002B7FF47E011277B6E55825E0F558755965
:1037AB0001E5582401FFE433FEC3E5599FEE648025
:1037BB00F874809840030238A1E55B2559F582E443
:1037CB00355AF583E0FFE55B2559F582E4355AF56B
:1037DB0083A3E0FD12741790001FE0FF30E006306A
:1037EB004903C22022EF30E106304D03C22122EF04
:1037FB0030E206305103C22222EF30E3063054038D
:10380B00C22322055905598098E5576402600302CB
:10381B0038A1C22BC22CC22DC22E7FF47E0112778F
:10382B00B6E55825E0F558755901E5582401FFE434
:10383B0033FEC3E5599FEE6480F87480985057E5CA
:10384B005B2559F582E4355AF583E0FFE55B255995
:10385B00F582E4355AF583A3E0FD12741790001F2F
:10386B00E030E005303902802290001FE030E105A6
:10387B00303A02801690001FE030E205303B0280A8
:10388B000A90001FE030E308303C05C220027105AE
:06389B0005590559809457
:0138A1002204
:0241B0008F4D31
:1041B200C2659000A8E0FFE54DB401167868E6FEFE
:1041C200D39F400EEE9FF55074102FF582E4341BFE
:1041D200804FE54DB402167869E6FED39F400EEE9D
:1041E2009FF55074602FF582E4341B8034E54DB4A2
:1041F2000316786AE6FED39F400EEE9FF55074B028
:104202002FF582E4341B8019E54DB4041C786BE66B
:10421200FED39F4014EE9FF55074002FF582E434D4
:104222001CAF82F5518F52D2652065030242C0D283
:1042320069AF4D1257C27FF47E011277B67D207F9F
:10424200051274177D1A7F081274177FC87E001238
:1042520077B6E4F54EE54EC39550505B0552E552F4
:10426200AE517002055114F5828E83E0F54F60362F
:1042720024F5601414601714601A14601D14602071
:1042820024057028E4FD80277D5F7F0780227D5E04
:104292007F06801C7D0A7F0280167D327F0280109D
:1042A2007D467F02800A7D0A7F038004AD4FE4FFD2
:0E42B200127417054E809EC269AF4D1257C29E
:0142C00022DB
:1074940030290F900671E0FF7C0B7D10126FD5B27E
:1074A4002922202912900670E0FF7C0A7DF0126FD9
:0874B400D5B229E4786CF62240
:105CE9007D3F7F091274177D507F08127417900049
:105CF9000EE493FDE4FF1274177D5B7F061274179F
:105D090090000FE493FDE4FF127417900010E493E0
:105D1900FDE4FF127417900011E49324BFB4080046
:105D29005053905D3975F003A4C58325F0C583737D
:105D3900025D51025D55025D59025D5F025D6502BA
:105D49005D6B025D71025D777D0A80067D3280029E
:105D59007D467F02801C7D0A7F0380167D287F0394
:105D690080107D467F03800A7D0A7F0480047D2898
:065D79007F0412741722E2
:10750C008F53D2691257C27D4B7F021274177D04C0
:10751C00E4FF1274177D387F04127417125CE9C2F1
:07752C0069AF531257C222A0
:0B774400855182855083E0FFA3E0FD2B
:10774F00BF0A02E4FFBD0A02E4FDEF75F00AA42DA3
:02775F00FF2207
:10518800C265D208D2207FF47E011277B67D2E7FC9
:10519800031274177D607F02127417C208C22012AE
:1051A80032027F081275A540030252543049F012AA
:1051B80032022049FA7868E6640770427E007F7000
:1051C80075331B7534108F828E837407F07D01E56B
:1051D800342DF582E43533F583E58224FFF582E545
:1051E8008334FFF583E0F9EF2DF582E43EF583E99A
:1051F800F00DBD08DAD2657F647E001277B67F08AD
:105208001275A5504720650302518AD208D2207F23
:10521800F47E011277B67D607F021274177D327FAB
:10522800061274177D1E7F05127417C208C2207CEF
:10523800007D707B087F787E001265117F081275EB
:10524800A550097F327E001277B680F01269D87FA8
:06525800647E001277B62F
:01525E00222D
:10746B00E4F53DC258C258F532302F05C22FC23F4A
:10747B0022303005C230C24122303105C231C24305
:09748B0022303204C232C2452253
:104098007580FFC286E580540FFFC285E580C45451
:1040A800F04FF520D2867D027F01125F2B40107DF4
:1040B800037F01125F2B4007300004D23980287D2E
:1040C800027F01125F2B500A300007300104D239F9
:1040D80080157D037F01125F2B500A2000033001F9
:1040E80004D2398002C2397D027F02125F2B401050
:1040F8007D037F02125F2B4007300204D23A8028EA
:104108007D027F02125F2B500A300207300304D26F
:104118003A80157D037F02125F2B500A200203307C
:104128000304D23A8002C23A7D027F03125F2B4019
:10413800107D037F03125F2B4007300404D23B80BD
:10414800287D027F03125F2B500A300407300504D4
:10415800D23B80157D037F03125F2B500A20040396
:10416800300504D23B8002C23B7D027F04125F2BE4
:10417800400F7D037F04125F2B4006300603D23CBC
:10418800227D027F04125F2B500930060630070398
:10419800D23C227D037F04125F2B50092006033096
:0741A8000703D23C22C23CD8
:0141AF0022ED
:10320200202B6A20391C205019901CFAE07002A36E
:10321200E0700B7D067F01125F2B5002D247C2493C
:10322200804B30392130501E901CE0E07002A3E048
:10323200700B7D087F01125F2B5002D23D3063027A
:10324200D259D24980273039082050051269D880D6
:103252001C203919305016C249C250C214C210C2C1
:103262001CC2181276D07868E66002D259202C71FE
:10327200203A1C205319901CFCE07002A3E0700B52
:103282007D067F02125F2B5002D24BC24D8052301C
:103292003A28305325901CE2E07002A3E070127DC0
:1032A200087F02125F2B50097F021275335002D23F
:1032B2003E306402D259D24D8027303A082053055D
:1032C200126A2C801C203A19305316C24DC253C2C6
:1032D20015C211C21DC2191276ED7869E66002D2DA
:1032E2005A202D71203B1C205519901CFEE07002C3
:1032F200A3E0700B7D067F03125F2B5002D24EC2F9
:10330200518052303B28305525901CE4E07002A3D6
:10331200E070127D087F03125F2B50097F03127544
:10332200335002D240302802D259D2518027303B4A
:1033320008205505126A80801C203B19305516C2A0
:1033420051C255C216C212C21EC21A12770A786A36
:10335200E66002D25B202E6D203C1B205618901D89
:1033620000E07002A3E0700B7D067F04125F2B5019
:1033720002D252C25422303C27305624901CE6E03E
:103382007002A3E070127D087F04125F2B50097F48
:10339200041275335002D242302A02D259D2542238
:1033A200303C06205603026AD4203C19305616C21D
:1033B20054C256C217C213C21FC21B127727786BA0
:0633C200E66002D25E226B
:04790900124EE02218
:104EE00090001FE0540FFFBF010B304906203D0327
:104EF000024FA7C322EF64037014304906203D031C
:104F0000024FA7304D06203E03024FB2C322EF648A
:104F1000057014304906203D03024FA7305106208A
:104F20004003024FBDC322EF6409701330490520CE
:104F30003D028073305406204203024FC8C322EF63
:104F40006407701A304905203D02805B304D052012
:104F50003E02805E3051052040028061C322EF6432
:104F60000B701A304905203D02803C304D05203E33
:104F700002803F305405204202804DC322EF640D71
:104F8000701A304905203D02801D30510520400235
:104F9000802B305405204202802EC322EF640F7014
:104FA0002E304908203D05753E01D322304D0820A2
:104FB0003E05753E02D322305108204005753E0360
:104FC000D322305408204205753E04D322C322C3A5
:014FD00022BE
:10753300BF010690001FE01322BF020790001FE067
:10754300A2E122BF030790001FE0A2E222BF0406CC
:0775530090001FE0A2E322FB
:1069D8007868E6602275331B753410E4FFE5342FC0
:1069E800F582E43533F583E4F00FBF50F075331BBF
:1069F800753410E47868F6900600E0FFA3E0901C78
:106A0800E0CFF0A3EFF0900608E0FFA3E0901CFAB7
:106A1800CFF0A3EFF0C246C247C25DC23DC263C217
:036A28003FD2500A
:016A2B002248
:106A2C007869E6602275351B753660E4FFE5362F14
:106A3C00F582E43535F583E4F00FBF50F075351B66
:106A4C00753660E47869F6900602E0FFA3E0901CCE
:106A5C00E2CFF0A3EFF090060AE0FFA3E0901CFC5D
:106A6C00CFF0A3EFF0C248C24BC25FC23EC264C2B9
:036A7C0041D253B1
:016A7F0022F4
:106A8000786AE6602275371B7538B0E4FFE5382F69
:106A9000F582E43537F583E4F00FBF50F075371B0E
:106AA0007538B0E4786AF6900604E0FFA3E0901C25
:106AB000E4CFF0A3EFF090060CE0FFA3E0901CFE03
:106AC000CFF0A3EFF0C24CC24EC260C240C228C297
:036AD00043D25559
:016AD30022A0
:106AD400786BE6602275391C753A00E4FFE53A2FBD
:106AE400F582E43539F583E4F00FBF50F075391CB5
:106AF400753A00E4786BF6900606E0FFA3E0901C7C
:106B0400E6CFF0A3EFF090060EE0FFA3E0901D00A7
:106B1400CFF0A3EFF0C24FC252C261C242C22AC236
:036B240045D25601
:016B2700224B
:10570D00C208C209C20EC20C12779AC265D25CE4FD
:10571D00F53D7FE87E031277B6C298C2AF75567F0E
:10572D00755596755498755300785374FF1256EF4E
:10573D00E4FBFAF9F8C31256DC504430983E1200DF
:10574D00061278CBEF14601824F0602624C1600B8C
:10575D0024F670287F061278F98021126E79801C4C
:10576D007F061278F9127210127393126CBCD26507
:10577D00800A7F061278F91264A0D2653065AAE41A
:10578D00786CF6D2697F011257C27F011268D87DFD
:10579D00467F021274177D1E7F071274177D147FCA
:1057AD00081274177D327F03127417C2697F0112BC
:0457BD0057C2C25CB1
:0157C10022C5
:1064A000756701756500756620E4F5577F021278FF
:1064B000F9E5672402F559AF671278F9E4F558E574
:1064C000662558F582E43565F583E0FF1278F9E535
:1064D000662558F582E43565F583E02559F55905BB
:1064E00058E558C3948040D7AF591278F97F03120A
:1064F00078F9127901EF64156016056774802566D6
:10650000F566E43565F5650557E557C39435409C58
:016510002268
:10721000756701756500756620E4F5571273665051
:10722000077F061278F980057F150278F9056774E3
:10723000802566F566E43565F5650557E557C39421
:037240003540D9FD
:017243002228
:10736600E4F55812790174502558F582E4341CF579
:1073760083EFF00558E558C3948440E712783190BE
:0C7386001CD2E0B50705127635D322C3F7
:0173920022D8
:10763500E4FF74522FF582E4341CF583E0FEE56621
:0F7645002FF582E43565F583EEF0000FBF80E38B
:017654002213
:10783100E4FFFE74502EF582E4341CF583E02FFF43
:047841000EBE82EF06
:017845002220
:106E7900E4F557F55D755CE0755B93755A04F55952
:106E8900785974FF1256EFE4FBFAF9F8C31256DC8D
:106E990050253098EB1200068F58E55864046017A6
:106EA900AF5D055D74502FF582E4341CF583E55818
:076EB900F02557F55780C9D1
:016EC00022AF
:04000600AF99C29854
:01000A0022D3
:0878F9003099FDC2998F99221C
:077901003098FDAF99C29818
:01790800225C
:10592A000701020304050607070706050403020127
:10593A0003010A0A03020A0A03030A0A03040A0AF7
:10594A00030307050303020503070A0A04024B00BF
:10595A00040438072E03024B0004043802055F00D2
:10596A000302055F000402055F000502055F0006E9
:10597A0002055F000702055F000802055F000902D1
:10598A00055F000A02055F000B02055F000C0205B5
:10599A005F000D02055F000E02055F000F02055F42
:1059AA00001002055F001102055F001204072E08AD
:1059BA00260640033204072E082606400253080C26
:0759CA000A1D040000241B6C
:10001600C2AF9000207491F09000217481F090009E
:1000260022F0900023F09000247403F090002574D1
:10003600BFF09000267408F0900027740FF090002F
:10004600307409F0A37403F0E4A3F0A37410F0A3D2
:100056007403F0E4A3F0A37415F0A37403F0A3747F
:1000660015F0A37403F0E4A3F0A37410F0A37403D3
:10007600F0E4A3F0A37409F0A37403F07E597F3A69
:100086007C007D807B04126F947E597F3E7C007DD0
:10009600887B04126F947E597F427C007D907B049E
:1000A600126F947E597F467C007D987B04126F9474
:1000B6007E597F4E7C007DA07B04126F947E597F13
:1000C6004A7C007DA87B04126F947E597F527C0087
:1000D6007DB07B04126F947E597F2A7C007D707BF5
:1000E60008126F947E597F327C007D787B08126FF0
:1000F600947E597F567C037D807B09126F947E59CE
:100106007F5F7C037DA07B07126F947E597F667CA0
:10011600037DC07B05126F947E597F6B7C037DE067
:100126007B05126F947E597F707C047D007B0512DF
:100136006F947E597F757C047D207B05126F947EBB
:10014600597F7A7C047D407B05126F947E597F7FB0
:100156007C047D607B05126F947E597F847C047DD0
:10016600807B05126F947E597F897C047DA07B0578
:10017600126F947E597F8E7C047DC07B05126F942E
:100186007E597F937C047DE07B05126F947E597FB8
:10019600987C057D007B05126F947E597F9D7C05BA
:1001A6007D207B05126F947E597FA27C057D407B66
:1001B60005126F947E597FA77C057D607B05126FC3
:1001C600947E597FAC7C057D807B05126F947E59A9
:1001D6007FB17C057DA07B05126F947E597FB67C2E
:1001E600057DC07B09126F947E597FBF7C057DE03B
:1001F6007B09126F94900600E4F0A374B4F09006A5
:1002060002E4F0A374B4F0900604E4F0A374B4F02E
:10021600900606E4F0A374B4F09006187401F0A3F7
:1002260074E0F090061AE4F0A37478F090061EE4E9
:10023600F0A3743CF09006087402F0A37458F09092
:10024600060A7402F0A37458F090060C7402F0A328
:100256007458F090060E7402F0A37458F074079068
:100266000610F0A3F0900612F0A3F0900614F0A387
:10027600F0900616F0A3F0900620F0A3F090062268
:10028600F0A3F090061C7402F0A37458F0900630A8
:10029600740AF09006317428F0900633740AF090D0
:1002A6000634F09006327405F07E597FC87C067DD0
:1002B600407B09126F9490063D7417F090063E74C9
:1002C6000CF090063C7419F0E490063FF090063B63
:1002D600740CF09006527401F09007307469F0A324
:1002E6007411F09006537401F09007507469F0A3EE
:1002F6007410F09006547401F09007707469F0A3BE
:100306007421F09006557401F09007907469F0A37B
:100316007420F09006567401F09007B07469F0A34B
:100326007431F09006577401F09007D07469F0A309
:100336007430F09006587401F09007F07469F0A3D9
:100346007441F09006597401F09008107469F0A396
:100356007440F090065A7401F09008307462F0A36D
:100366007411F0A37432F0A37401F0A37450F0A3D7
:100376007410F090065B7401F09008507461F0A35D
:100386007420F0A37462F0A37411F0A37432F0A386
:100396007402F0A37450F0A37410F090065C74011C
:1003A600F09008707451F0A37411F0A37433F0A3A5
:1003B600E4F0A37451F0A37410F090065D7401F09C
:1003C6009008907462F0A37411F0A37430F0A374D3
:1003D60002F0A37462F0A37410F090065E7401F04C
:1003E6009008B07451F0A37411F0A37441F0A37493
:1003F60010F0A37451F0A37410F090065F7401F02E
:100406009008D07451F0A37411F0A37434F0A3745F
:1004160014F0A37451F0A37410F09006607401F008
:100426009008F07451F0A37411F0A37434F0A3741F
:1004360018F0A37451F0A37410F09006617401F0E3
:100446009009107451F0A37411F0A37434F0A374DE
:1004560028F0A37451F0A37410F09006627401F0B2
:100466009009307462F0A37411F0A37430F0A37491
:1004760003F0A37462F0A37410F09006637401F0A5
:100486009009507462F0A37411F0A37430F0A37451
:1004960004F0A37462F0A37410F09006647401F083
:1004A6009009707462F0A37411F0A37460F0A374E1
:1004B60001F0A37495F0A3743DF0A37490F0A374B7
:1004C60001F0A37498F0A37426F0A37496F0A374B5
:1004D60040F0A37462F0A37410F0A37461F0A374E7
:1004E60070F09006657401F09009907462F0A37440
:1004F60011F0A37460F0A37401F0A37495F0A374D3
:100506003DF0A37490F0A37401F0A37496F0A37465
:1005160038F0A37462F0A37410F09006667401F0CC
:100526009009B07462F0A37411F0A37460F0A37420
:1005360001F0A37495F0A3743DF0A37490F0A37436
:1005460002F0A37498F0A37426F0A37496F0A37433
:1005560040F0A37462F0A37410F0A37461F0A37466
:1005660070F09006677401F09009D07462F0A3747D
:1005760011F0A37460F0A37401F0A37495F0A37452
:100586003DF0A37490F0A37402F0A37496F0A374E4
:1005960038F0A37462F0A37410F09006687401F04A
:1005A6009009F07462F0A37411F0A37460F0A37460
:1005B60001F0A37495F0A3743DF0A37490F0A374B6
:1005C60003F0A37498F0A37426F0A37496F0A374B2
:1005D60040F0A37462F0A37410F0A37461F0A374E6
:1005E60070F09006697401F0900A107462F0A374BA
:1005F60011F0A37460F0A37401F0A37495F0A374D2
:100606003DF0A37490F0A37403F0A37496F0A37462
:1006160038F0A37462F0A37410F090066A7401F0C7
:10062600900A307462F0A37411F0A37460F0A3749E
:1006360001F0A37495F0A3743DF0A37490F0A37435
:1006460004F0A37498F0A37426F0A37496F0A37430
:1006560040F0A37462F0A37410F0A37461F0A37465
:1006660070F090066B7401F0900A507462F0A374F7
:1006760011F0A37460F0A37401F0A37495F0A37451
:100686003DF0A37490F0A37404F0A37496F0A374E1
:1006960038F0A37462F0A37410F09006707401F041
:1006A600900AF07464F0A37411F0A37496F0A37426
:1006B60032F0A37495F0A3741EF0A37498F0A3749B
:1006C6004BF0A37464F0A37410F09006717401F0FB
:1006D600900B107464F0A37411F0A37496F0A374D5
:1006E60032F0A37495F0A3741EF0A37493F0A37470
:1006F60018F0A37464F0A37410F09006737401F0FC
:10070600900B507462F0A37411F0A37460F0A3749C
:1007160001F0A37495F0A3743DF0A37490F0A37454
:1007260002F0A37497F0A37426F0A37493F0A37455
:1007360018F0A37462F0A37410F0A37470F0A3749D
:1007460010F09006747401F0900B707462F0A3744C
:1007560011F0A37460F0A37401F0A37495F0A37470
:100766003DF0A37490F0A37403F0A37497F0A37400
:1007760026F0A37493F0A37418F0A37462F0A37424
:1007860010F0A37470F0A37420F09006757401F055
:10079600900B907462F0A37411F0A37460F0A374CC
:1007A60001F0A37495F0A3743DF0A37490F0A374C4
:1007B60004F0A37497F0A37426F0A37493F0A374C3
:1007C60018F0A37462F0A37410F0A37470F0A3740D
:1007D60030F09006817401F0900D107462F0A374ED
:1007E60011F0A37460F0A37401F0A37492F0A374E3
:1007F6004BF0A37490F0A37404F0A37494F0A37464
:1008060038F07499A3F0A3F0A37460F0A37401F018
:10081600A37462F0A37410F01221DC126CBCD269CE
:100826007F011257C27D2F7F071274177D0C7F033D
:100836001274177D327F061274177D1E7F0512749F
:100846001790001F7401F0FD7F1F7E00127015C205
:07085600697F011257C22265
:1021DC009001007402F0A3740DF0A37402F0900649
:1021EC00A014F09010F07464F0A37411F0A3749721
:1021FC00F0A3742EF0A37495F0A3743DF0A3749027
:10220C00F0A37402F0A37496F0A37438F0A3746472
:10221C00F0A37410F0A37470F0A37411F090010883
:10222C007402F0A3740EF0A37402F09006A114F0E3
:10223C009011107464F0A37411F0A37497F0A3744C
:10224C002EF0A37495F0A3743DF0A37490F0A374D6
:10225C0002F0A37496F0A37436F0A37464F0A37424
:10226C0010F0A37470F0A37410F09001107402F0CD
:10227C00A3740DF0A37403F09006A27401F09011F6
:10228C00307464F0A37411F0A37497F0A3742EF05F
:10229C00A37495F0A3743DF0A37490F0A37403F0B1
:1022AC00A37496F0A37438F0A37464F0A37410F0C4
:1022BC00A37470F0A37421F09001187402F0A3744D
:1022CC000EF0A37403F09006A37401F090115074F7
:1022DC0064F0A37411F0A37497F0A3742EF0A3749C
:1022EC0095F0A3743DF0A37490F0A37403F0A37461
:1022FC0096F0A37436F0A37464F0A37410F0A37476
:10230C0070F0A37420F09001207402F0A3740DF00F
:10231C00A37404F09006A47401F09011707464F02E
:10232C00A37411F0A37497F0A3742EF0A37495F01A
:10233C00A3743DF0A37490F0A37404F0A37496F00E
:10234C00A37438F0A37464F0A37410F0A37470F049
:10235C00A37431F09001287402F0A3740EF0A374EE
:10236C0004F09006A57401F09011907464F0A374BD
:10237C0011F0A37497F0A3742EF0A37495F0A374CA
:10238C003DF0A37490F0A37404F0A37496F0A374BE
:10239C0036F0A37464F0A37410F0A37470F0A374FB
:1023AC0030F09001307403F0A3740DF0A37402F0BC
:1023BC00A304F09006A67401F09011B07464F0A31D
:1023CC007411F0A37497F0A3742EF0A37495F0A37A
:1023DC00743DF0A37490F0A37402F0A37490F0A376
:1023EC007403F0A37496F0A37438F0A37464F0A390
:1023FC007410F0A37470F0A37441F090013874035E
:10240C00F0A3740EF0A37402F0A304F09006A7746A
:10241C0001F09011D07464F0A37411F0A37497F0D0
:10242C00A3742EF0A37495F0A3743DF0A37490F0F4
:10243C00A37402F0A37490F0A37403F0A37496F049
:10244C00A37436F0A37464F0A37410F0A37470F04A
:10245C00A37440F09001407404F0A3740DF0A374C5
:10246C0002F0A304F0A304F09006A87401F09011FC
:10247C00F07464F0A37411F0A37497F0A3742EF0AD
:10248C00A37495F0A3743DF0A37490F0A37402F0C0
:10249C00A37490F0A37403F0A37490F0A37404F0ED
:1024AC00A37496F0A37438F0A37464F0A37410F0C2
:1024BC00A37470F0A37441F0A37470F0A37451F082
:1024CC009001487404F0A3740EF0A37402F0A304FA
:1024DC00F0A304F09006A97401F09012107464F04B
:1024EC00A37411F0A37497F0A3742EF0A37495F059
:1024FC00A3743DF0A37490F0A37402F0A37490F055
:10250C00A37403F0A37490F0A37404F0A37496F076
:10251C00A37436F0A37464F0A37410F0A37470F079
:0D252C00A37440F0A37470F0A37450F0226B
:0A6F94008E4C8F4D8C4E8D4F8B50AC
:106F9E00E4F9C3E5506480F8E96480985028E9FF6D
:106FAE003395E0FEE54D2FF582E54C3EF583E493F7
:106FBE00FFE9FD3395E0FCE54F2DF582E54E3CF5FE
:066FCE0083EFF00980CC06
:016FD400229A
:1077EB00D291C2A4C2A5C2A6C2A7007F0512781B64
:0977FB000012780500D2A7D2911A
:017804002261
:107694001277EBEF20E0F9D291C2A4C2A5C2A6C230
:0E76A400A7007F0612781B0000D2A7D2912209
:1076B2001277EBEF20E0F9D291C2A4C2A5C2A6C212
:0E76C200A7007F0412781B0000D2A7D29122ED
:046B28008E528F53A7
:106B2C00AE04AF058E568F57D291C2A4C2A5C2A691
:106B3C00C2A7007F0312781BE552FF12781BAF53DC
:106B4C0012781BE4F554F555127805E5572555F5E3
:106B5C0082E5563554F583EFF00555E55570020581
:0E6B6C0054C39420E554940040DED2A7D29189
:016B7A0022F8
:08664F008E5D8F5E8C5F8D6093
:106657001277EBEF20E0F9127694855D63855E642F
:10666700D291C2A4C2A5C2A6C2A7007F0212781BFC
:10667700E55FFF12781BAF6012781BE4F561F562E6
:10668700E5642562F582E5633561F583E0FF1278FD
:106697001B0562E56270020561C39420E561940001
:0766A70040DE00D2A7D291F2
:0166AE0022C9
:0A6511008E4C8F4D8C4E8D4F8B5039
:10651B00C2AF1276941277EBEF20E0F9854E5285DD
:10652B004F53D291C2A4C2A5C2A6C2A7007F02122A
:10653B00781BE54CFF12781BAF4D12781BE4F5511D
:10654B00AF50EF3395E0FEC3E5519FEE6480F874D6
:10655B0080985014E5532551F582E43552F583E0CC
:10656B00FF12781B055180D800D2A7D2911276B2B8
:02657B00D2AF9D
:01657D0022FB
:107015008E5B8F5C8D5DC2AF1276941277EBEF209D
:10702500E0F9D291C2A4C2A5C2A6C2A7007F0212EE
:10703500781BE55BFF12781BAF5C12781BAF5D1206
:0E704500781B0000D2A7D2911276B2D2AF22F1
:04755A008E4C8F4D77
:10755E00D291C2A4C2A5C2A6C2A77F0312781BE510
:10756E004CFF12781BAF4D12781B127805D2A7D2A2
:01757E00917B
:01757F0022E9
:106EC100C2AF754E00754F20755000755120E4F525
:106ED1004CF54DAD4FAC4EAF51AE50126B287420F6
:106EE100254FF54FE4354EF54E74202551F551E40B
:106EF1003550F550054DE54D7002054CC394D6E56E
:076F01004C940040CED2AF1A
:016F08002266
:106CBC00C2AF755B00755C20755900755A20E4F500
:106CCC0057F558AD5AAC59AF5CAE5B12664F742099
:106CDC00255AF55AE43559F5597420255CF55CE4D0
:106CEC00355BF55B0558E55870020557C394D6E53E
:0A6CFC0057940040CE1276B2D2AFDA
:016D0600226A
:046BCD008C4D8D4E10
:106BD100EF6048D22BD22CD22DD22EE4F54F854E28
:106BE10082854D83E0FEA3E04E6028AF4FEF3395E1
:106BF100E0FEEF25E0FFEE33FEE54E2FF582E54D99
:106C0100125334926520650B054FC3E54F648094A0
:0B6C11009040CBC22BC22CC22DC22E23
:016C1C002255
:046FD5008C4D8D4E04
:106FD900EF6038E4F54F854E82854D83E0FEA3E0EE
:106FE9004E6028AF4FEF3395E0FEEF25E0FFEE331B
:106FF900FEE54E2FF582E54D125334926520650B5F
:0B700900054FC3E54F6480949040CB1E
:017014002259
:085334003EF583E0FEA3E0FF5B
:04533C00AD07AC0607
:10534000C266780CEF088006A2E0CE13CE13D8F820
:10535000540FF5507808AF05AE04EF088006A2E0C0
:10536000CE13CE13D8F8540FF5517804AF05AE0420
:10537000EF088006A2E0CE13CE13D8F8540FF552F2
:10538000ED540FF553E550607CB4010BAB53AD52B7
:10539000AF51125597806EE550B4030BAB53AD522D
:1053A000AF511267CA805EE550B4040BAB53AD52E7
:1053B000AF51126D07804EE550B4050BAB53AD52A3
:1053C000AF51123A2B803EE550B4060BAB53AD52B1
:1053D000AF511216F3802EE550B4070BAB53AD520C
:1053E000AF5112525F801EE550B4080BAB53AD5263
:1053F000AF51126B7B800EE550B40909AB53AD522F
:07540000AF511275CAA2664C
:015407002282
:105597008F548D558B56E554B40113900020E0FFCE
:1055A700126772900020EFF0FD7F20025632E5541B
:1055B700B4021190002112676C900021EFF0FD7F7B
:1055C70021025632E554B4031090002212676C9002
:1055D7000022EFF0FD7F228052E554B404109000C2
:1055E7002312676C900023EFF0FD7F23803DE55485
:1055F700B4051090002412676C900024EFF0FD7F33
:10560700248028E554B4061090002512676C90009A
:1056170025EFF0FD7F258013E554B407139000268E
:1056270012676C900026EFF0FD7F267E0002701552
:10563700E554B4081690002712676C900027EFF026
:0C564700FD7F277E001270151273932265
:06676C00E0FFAB56AD5545
:10677200D267AC07BD01047E018033BD02047E02F4
:10678200802CBD03047E048025BD04047E08801E87
:10679200BD05047E108017BD06047E208010BD0753
:1067A200047E408009BD08047E808002C267BB016E
:1067B20005EE4204800BEB7006EEF452048002C236
:0767C20067306703AF0422FA
:0167C90022AD
:1067CA008F548D558B56E554700BAD56AF551278D4
:1067DA00ABE4FD801EE554B4010BAD56AF551278FB
:1067EA00AB7D01800EE554B4020CAD56AF5512785C
:1067FA00AB7D02023719E554B4030AE55570061257
:10680A007105C25822E554B40410AD56AF5512644E
:0B681A006E8F3F753D05E53D70FC22D0
:106D07008F548D558B56E5547027E555B401047D96
:106D1700018019E555B402047D028010E555B403DE
:106D2700047D038007E555B404207D04AF56026F48
:106D370009E554B40114E555D39400400DE5559485
:0B6D4700055007753D01E53D70FC2282
:103A2B008B54EF7017BD0114E5547002C220E5549E
:103A3B0064016003023B97D220023B97EF7017BDE6
:103A4B000214E5547002C221E55464016003023B89
:103A5B0097D221023B97EF7017BD0314E554700208
:103A6B00C222E55464016003023B97D222023B97CA
:103A7B00EF7017BD0414E5547002C223E5546401C2
:103A8B006003023B97D223023B97EF701BBD0518D7
:103A9B00E5547004C220C221E55464016003023B6B
:103AAB0097D220D221023B97EF701BBD0618E5542D
:103ABB007004C222C223E55464016003023B97D217
:103ACB0022D223023B97BF0117BD0114E5547002AC
:103ADB00C224E55464016003023B97D224023B9756
:103AEB00BF0117BD0214E5547002C225E5546401F1
:103AFB006003023B97D225023B97BF0116BD031310
:103B0B00E5547002C226E55464016003023B97D270
:103B1B00268079BF0113BD0410E5547002C227E55E
:103B2B005464017067D2278063BF0117BD0514E58C
:103B3B00547004C224C225E5546401704FD224D2C0
:103B4B00258049BF0117BD0614E5547004C226C277
:103B5B0027E55464017035D226D227802FEF6401FC
:103B6B00702AED64097025E554B401047F018019B6
:103B7B00E554B402047F028010E554B403047F03C0
:103B8B008007E554B404057F041268D87F327E00A9
:043B9B001277B622C5
:1016F3008F548D558B56E5547016AD56AF551278F1
:10170300AB901D14EFF0901D14E0D3940050F7221A
:10171300E554B40117E555B40112E5567002C20849
:10172300E55664016003021A99D20822E554B40114
:1017330017E555B40212E5567002C209E556640175
:101743006003021A99D20922E554B40117E555B48E
:101753000312E5567002C20EE55664016003021AD5
:1017630099D20E22E554B40117E555B40412E55697
:101773007002C20CE55664016003021A99D20C226E
:10178300E554B4011BE555B40516E5567004C208CB
:10179300C209E55664016003021A99D208D20922EC
:1017A300E554B40118E555B40613E5567004C20EAA
:1017B300C20CE55664016003021A998024E554645F
:1017C300017023E555B4071EE5567008C208C20927
:1017D300C20EC20CE55664016003021A99D208D204
:1017E30009D20ED20C22E554B4021DE555B40118FA
:1017F300E5567004C208C220E55664016003021A6C
:1018030099D208D2200219B9E554B4021DE555B4A2
:101813000218E5567004C209C221E556640160034B
:10182300021A99D209D221021945E554B4021DE5E1
:1018330055B40318E5567004C20EC222E55664017E
:101843006003021A99D20ED222021969E554B40236
:101853001DE555B40418E5567004C20CC223E556C1
:1018630064016003021A99D20CD22302198CE55445
:1018730064027026E55564057020E5567008C208B9
:10188300C209C220C221E55664016003021A99D23B
:1018930008D209D220D2210219B9E5546402702674
:1018A300E55564067020E5567008C20EC20CC222CC
:1018B300C223E55664016003021A99D20ED20CD2F8
:1018C30022D223021969E55464027035E555640791
:1018D300702FE5567010C208C209C20EC20CC22096
:1018E300C221C222C223E55664016003021A99D2BF
:1018F30008D209D20ED20CD220D221D222D22380F6
:1019030065E554B4031DE555B40118E5567004C2EA
:1019130008C224E55664016003021A99D208D2244E
:101923000219B9E554B4031FE555B4021AE556701C
:1019330004C209C225E55664016003021A99D2095B
:10194300D2257F020219E8E554B4031EE555B4031A
:1019530019E5567004C20EC226E5566401600302FF
:101963001A99D20ED2267F03807BE554B4031EE579
:1019730055B40419E5567004C20CC227E556640138
:101983006003021A99D20CD2277F048058E554646D
:10199300037027E55564057021E5567008C208C237
:1019A30009C224C225E55664016003021A99D208CC
:1019B300D209D224D2257F01802BE55464037028F9
:1019C300E55564067022E5567008C20EC20CC226A5
:1019D300C227E55664016003021A99D20ED20CD2D3
:1019E30026D2277F030268D8E554B4040AE555B428
:1019F3000105AF56026334E554B4040AE555B40255
:101A030005AF560265E7E5546409701EE555B40158
:101A130019E5567003C20A22E556B40103D20A221D
:101A2300E556640270707F058069E5546409701E91
:101A3300E555B40219E5567003C20B22E556B4010D
:101A430003D20B22E5566402704C7F068045E554B1
:101A53006409701EE555B40319E5567003C20F22DD
:101A6300E556B40103D20F22E556640270287F07BE
:101A73008021E5546409701EE555B40419E55670D8
:101A830003C20D22E556B40103D20D22E556B4027A
:071A9300057F08125D7F22B0
:10525F00AC07EC6003025315BD010CEB7009900015
:10526F001FE054FDF0800DBD010ABB010790001F28
:10527F00E04403F0BD020CEB700990001FE054FBFB
:10528F00F0800DBD020ABB010790001FE04405F03E
:10529F00BD030CEB700990001FE054F7F0800DBDBB
:1052AF00030ABB010790001FE04409F0BD040CEB9B
:1052BF00700990001FE054F9F0800DBD040ABB0186
:1052CF000790001FE04407F0BD050CEB700990003C
:1052DF001FE054F3F0800DBD050ABB010790001FBE
:1052EF00E0440DF0BD060CEB700990001FE054F187
:1052FF00F08025ED64067020EB6401701B90001F99
:10530F00E0440FF08012BC010FED700CEB7004C283
:10531F00298005BB0102D22990001FE0FD7F1F7E6F
:05532F000012701522C0
:106B7B008F548D558B56E554700C1278A7744F2F8C
:106B8B00F58274068020E554B4010C1278A7744F7B
:106B9B002FF58274068024E554B402101278A77482
:106BAB009F2FF58274063EF583E4F022E554B4037F
:106BBB00101278A7749F2FF58274063EF58374012B
:026BCB00F022B6
:0275CA008F54DC
:1075CC00AF057804EF08800123D8FD4BF555E55441
:1075DC00B40908E555B49903025CE9AD55AF5412F2
:0275EC00741712
:0175EE00227A
:10633400E545B40109BF0106D220D2088060E545D5
:10634400B40109EF7006C220C2088052E545B402C8
:1063540009BF0106D221D2098044E545B40209EF00
:106364007006C221C2098036E545B40309BF01069F
:10637400D222D20E8028E545B40309EF7006C2226A
:10638400C20E801AE545B40409BF0106D223D20C1B
:10639400800CE545B40407EF7004C223C20C1277E5
:0A63A4009AAF3E1268D812777E22ED
:1065E700E545B40108BF0105D224D20822E545B428
:1065F7000108EF7005C224C20822E545B40208BFAE
:106607000105D225D20922E545B40208EF7005C27B
:1066170025C20922E545B40308BF0105D226D20EDB
:1066270022E545B40308EF7005C226C20E22E545F0
:10663700B40408BF0105D227D20C22E545B40407EC
:08664700EF7004C227C20C220F
:0478A700AD56AF55D6
:0D78AB00EF75F00AA47C002DFFEC35F0FE17
:0178B80022AD
:02085D008F4DBD
:10085F00C266E4F53DD25CD2691257C27D4B7F026E
:10086F001274177D04E4FF1274177D387F0412741D
:10087F00177D607F0212741790061CE0FFA3E090B3
:10088F001CE8CFF0A3EFF0C269AF4D1257C2E4F5E9
:10089F0046C208123202E54DB40106A249926580A4
:1008AF001FE54DB40206A24D92658014E54DB403C9
:1008BF0006A25192658009E54DB40404A2549265D5
:1008CF00901CE8E07002A3E07005D266020EA7301C
:1008DF0065C1123202E54DB40106A2499265801F2F
:1008EF00E54DB40206A24D92658014E54DB40306A2
:1008FF00A25192658009E54DB40404A2549265207B
:10090F0065D0E54DB4010A754E1B754F10786880A0
:10091F002BE54DB4020A754E1B754F607869801C2C
:10092F00E54DB4030A754E1B754FB0786A800DE51F
:10093F004DB4040B754E1C754F00786BE6F550E502
:10094F0050D394005003020EA1854F82854E83E051
:10095F00640B6003020E9CA3E0FFB40A0AE550B4D7
:10096F000205D266020EA1EF64017032854F8285B7
:10097F004E83A3A3E064037025E550B40520854F93
:10098F0082854E83A3A3A3E0FFE54F2404F582E401
:10099F00354EF583E0FDAB4D123CF9020EA1854FAC
:1009AF0082854E83A3E0B40121854F82854E83A3B8
:1009BF00A3E0B40415E550D39405400EAB4DAD4FF5
:1009CF00AC4EAF501233C8020EA1854F82854E83B5
:1009DF00A3E064017032854F82854E83A3A3E06448
:1009EF00057025E550B40520854F82854E83A3A35E
:1009FF00A3E0FFE54F2404F582E4354EF583E0FDD7
:100A0F00AB4D12623A020EA1854F82854E83A3E051
:100A1F0064017032854F82854E83A3A3E064067014
:100A2F0025E550B40520854F82854E83A3A3A3E00F
:100A3F00FFE54F2404F582E4354EF583E0FDAB4D21
:100A4F001259D1020EA1854F82854E83A3E0B401C6
:100A5F0021854F82854E83A3A3E0B40715E550D3BC
:100A6F009405400EAB4DAD4FAC4EAF50124A08023D
:100A7F000EA1854F82854E83A3E064017032854FAE
:100A8F0082854E83A3A3E064087025E550B405204A
:100A9F00854F82854E83A3A3A3E0FFE54F2404F582
:100AAF0082E4354EF583E0FDAB4D126825020EA1B1
:100ABF00854F82854E83A3E0B40219854F82854E00
:100ACF0083A3A3E0B4080DE550B40308AF4D127330
:100ADF00EB020EA1854F82854E83A3E06402702442
:100AEF00854F82854E83A3A3E0B40818E550B40464
:100AFF0013854F82854E83A3A3A3E0FFAD4D1274E0
:100B0F00E4020EA1854F82854E83A3E0B4021985BE
:100B1F004F82854E83A3A3E0B4090DE550B40308BB
:100B2F00AF4D1273BF020EA1854F82854E83A3E096
:100B3F0064027024854F82854E83A3A3E0B4091805
:100B4F00E550B40413854F82854E83A3A3A3E0FF22
:100B5F00AD4D1274BC020EA1854F82854E83A3E06A
:100B6F0064037036854F82854E83A3A3E0640A70B9
:100B7F0029E55064057023854F82854E83A3A3A377
:100B8F00E0FFE54F2404F582E4354EF583E0FD12D6
:100B9F00774FAD4D1254D8020EA1854F82854E83EB
:100BAF00A3E06403703E854F82854E83A3A3E06468
:100BBF00017031E550D39405402A854F82854E83CD
:100BCF00A3A3A3E0FFE54F2404F582E4354EF5839C
:100BDF00E0FD12774F854D55AB50AD4FAC4E1242E5
:100BEF00C1020EA1854F82854E83A3E06403703648
:100BFF00854F82854E83A3A3E064027029E550647C
:100C0F00057023854F82854E83A3A3A3E0FFE54F95
:100C1F002404F582E4354EF583E0FD12774FAD4D98
:100C2F00126DE7020EA1854F82854E83A3E0B403B8
:100C3F0019854F82854E83A3A3E0B4030DE550B40D
:100C4F000308AF4D127053020EA1854F82854E835C
:100C5F00A3E0B40321854F82854E83A3A3E0B404A0
:100C6F0015E550D39403400EAB4DAD50AF4FAE4E84
:100C7F00125BB8020EA1854F82854E83A3E0B403A9
:100C8F0019854F82854E83A3A3E0B4050DE550B4BB
:100C9F000308AF4D1278B9020EA1854F82854E839E
:100CAF00A3E0B4031D854F82854E83A3A3E0B40652
:100CBF0011E550B4050CAD4DAF4FAE4E1270CC02D6
:100CCF000EA1854F82854E83A3E064037024854F68
:100CDF0082854E83A3A3E0B40718E550B4041385AF
:100CEF004F82854E83A3A3A3E0FFAD4D127655022D
:100CFF000EA1854F82854E83A3E0B4031D854F82DD
:100D0F00854E83A3A3E0B40811E550B4050CAD4D97
:100D1F00AF4FAE4E1272D9020EA1854F82854E8310
:100D2F00A3E064057022E550B4041D854F82854E03
:100D3F0083A3A3E0FF854F82854E83A3A3A3E0FD8A
:100D4F00AB4D122C3C020EA1854F82854E83A3E042
:100D5F00B40524E54F2404F582E4354EF583E0B461
:100D6F000B15E550D39405400EAB4DAD50AF4FAEC4
:100D7F004E1243D1020EA1854F82854E83A3E064AC
:100D8F00067022E550B4041D854F82854E83A3A3C0
:100D9F00E0FF854F82854E83A3A3A3E0FDAB4D12E9
:100DAF002539020EA1854F82854E83A3E0B4062418
:100DBF00E54F2404F582E4354EF583E0B40B15E5D9
:100DCF0050D39405400EAB4DAD50AF4FAE4E1230D9
:100DDF001A020EA1854F82854E83A3E0640970220B
:100DEF00854F82854E83A3A3E0B40A16E550B40461
:100DFF0011854F82854E83A3A3A3E0FF126D52028C
:100E0F000EA1854F82854E83A3E064097023854F21
:100E1F0082854E83A3A3E0B40117E550B404128575
:100E2F004F82854E83A3A3A3E0FFAD4D127277804F
:100E3F0061854F82854E83A3E0B40920854F82855B
:100E4F004E83A3A3E0B40214E550D39404400DAB3A
:100E5F0050AD4DAF4FAE4E1213488036854F828541
:100E6F004E83A3E064097025854F82854E83A3A32B
:100E7F00E0B40317E550B40412854F82854E83A367
:100E8F00A3A3E0FFAD4D126C1D80078000AF4D1284
:100E9F0077612066030208A2C258D269AF4D12577C
:100EAF00C27D607F021274177D327F03127417C2E6
:0F0EBF0069AF4D1257C2126CBCE4786CF6C25C7E
:010ECE002201
:0833C8008F518C528D538B5480
:1033D000855382855283A3A3A3E0FF8D828C83E56E
:1033E0008224041264658F55E555D394005003027E
:1033F0003569E55594294003023569E55164067045
:103400004FD269AF541257C27D527F05127417AF65
:1034100055124906E5532405F582E43552F583E05B
:10342000B40112749F2555F582E43406F5837401C6
:10343000F07D38800F749F2555F582E43406F583BE
:10344000E4F07D367F06127417C269AF540257C28A
:10345000E5532406F582E43552F583E0640B6003FE
:10346000023569E5532405F582E43552F583E0B46D
:103470000110749F2555F582E43406F5837401F03C
:10348000800D749F2555F582E43406F583E4F0E45D
:10349000FFFEE5532407F582E43552F583E5822EDD
:1034A000F582E43583F583E0B40B04AF0680040EA7
:1034B000BE08DFEF7003023569C39408400302358C
:1034C0006975F008E555A424F8F582E5F03400F5B7
:1034D00083EFF07E01EF2401FDE433FCEEC39DECAD
:1034E0006480F87480985036E5532406F582E435FC
:1034F00052F583E5822EF582E43583F583E0FD7590
:10350000F008E555A424F8F582E5F03400F583E5EC
:10351000822EF582E43583F583EDF00E80B7E55316
:103520002408F582E43552F583E5822FF582E435EF
:1035300083F583E0640B602DEF2408FEC3E5519E04
:10354000F55175F004125653AEF0EE701CE553249D
:1035500007FDE43552FC7E00ED2FFBEE3CFAAD5545
:103560007F011238A2D2688002C268AF541278EB91
:013570002238
:107613008E5CF55DAF5BEF3395E0FEE5592FF582A8
:08762300E5583EF583A3E0FFEA
:0A762B00EFD3940940037F002222F0
:0838A2008F568D578A588B598F
:1038AA00755B01E4F55AAF5BEF3395E0FEE5592FFE
:1038BA00F582E5583EF583E0FF6409706512762BC0
:1038CA00755C008F5DAE5C7804EF08800633CE33FA
:1038DA00CE92E0D8F8127613EF425DAE5CAF5D7817
:1038EA0008EF08800633CE33CE92E0D8F88E5CF526
:1038FA005DAF5BEF3395E0FEE5592FF582E5583E63
:10390A00F583A3A3E0FFE55BFD3395E0FCE5592DC4
:10391A00F582E5583CF583A3A3A3E0FD12774F0295
:10392A0039BDAF5BEF3395E0FEE5592FF582E558D7
:10393A003EF583E0FF12762B755C008F5DAE5C78F6
:10394A0004EF08800633CE33CE92E0D8F81276130D
:10395A00EF425DAE5CAF5D7804EF08800633CE338C
:10396A00CE92E0D8F88E5CF55DAF5BEF3395E0FE62
:10397A00E5592FF582E5583EF583A3A3E0FF1276B9
:10398A002BEF425DAE5CAF5D7804EF08800633CE64
:10399A0033CE92E0D8F88E5CF55DAF5BEF3395E0FD
:1039AA00FEE5592FF582E5583EF583A3A3A3E0FF70
:1039BA0012762BEF425DE556701EAF5AEF3395E053
:1039CA00FEEF25E0FFEE33FE75F020E557A424D084
:1039DA00F582E5F034068021E556B4012FAF5AEF9F
:1039EA003395E0FEEF25E0FFEE33FE75F020E55754
:1039FA00A424D0F582E5F03410F583E5822FF58210
:103A0A00E5833EF583E55CF0A3E55DF07404255B90
:103A1A00F55B055AC3E55A6480949050030238B0A6
:013A2A002279
:084A08008F518C528D538B5429
:104A1000855382855283A3A3A3E0FF8D828C83E517
:104A20008224041264658F55E555D3940050030227
:104A30004AF5E55594334003024AF5E551640670A2
:104A40004FD269AF541257C27D527F05127417AF0F
:104A500055124906E5532405F582E43552F583E005
:104A6000B40112744F2555F582E43406F5837401C0
:104A7000F07D38800F744F2555F582E43406F583B8
:104A8000E4F07D367F06127417C269AF540257C234
:104A9000E5532406F582E43552F583E0640B705546
:104AA000E5532405F582E43552F583E0B401107432
:104AB0004F2555F582E43406F5837401F0800D74BA
:104AC0004F2555F582E43406F583E4F074F9255159
:104AD000F55175F004125653AFF0EF7014E55324FE
:104AE00006FBE43552FAAD55E4FF1238A2D26880D5
:104AF0000DC2688009C269AF541257C2C268AF5470
:034B00001278EB3D
:014B0300228F
:023CF9008B51ED
:103CFB0012646E8F54E554D394005003023E36E5A4
:103D0B005494334003023E36D269AF511257C27DF1
:103D1B00527F05127417AF54124906749F2554F540
:103D2B0082E43406F583E060047D3880027D367FC3
:103D3B00061274177F2C7E011277B675F008E554C6
:103D4B00A424F8F582E5F03400F583E0F552700712
:103D5B007D1B7F061274177D577F02127417E55275
:103D6B00607A755301AF52EF3395E0FEEF2401FFFC
:103D7B00E43EFEAD53ED3395E0FCC3ED9FEE648066
:103D8B00F8EC6480985055AF53EF3395E0FE75F027
:103D9B0008E554A424F8F582E5F03400F583E582B8
:103DAB002FF582E5833EF583E0B40A04E4FD80241D
:103DBB00AF53EF3395E0FE75F008E554A424F8F506
:103DCB0082E5F03400F583E5822FF582E5833EF53D
:103DDB0083E0FDE4FF127417055380897F2C7E016D
:103DEB001277B675F020E554A424D0F582E5F034B3
:103DFB0010F583E0FEA3E0FF900000EEF0A3EFF0E0
:103E0B004E70077D1B7F061274177D0C7F03127497
:103E1B0017900000E07002A3E06009E55414FD7FE9
:103E2B0001122E30C269AF510257C2C268AF511294
:023E3B0078EB22
:013E3D002262
:042E30008F558D56D7
:102E3400E4F557E5556003022EDBAF57EF3395E019
:102E4400FEEF25E0FDEE33FCAF56EF3395E0FEEFE9
:102E54007805C333CE33CED8F924F0F58274063E18
:102E6400F583E5822DF582E5833CF583E0FAA3E062
:102E7400FB780CFFAE02088006A2E0CE13CE13D876
:102E8400F8540FF5587808AF03AE02EF088006A295
:102E9400E0CE13CE13D8F8540FF559AF56EF33954F
:102EA400E0FEEF7805C333CE33CED8F924F0F582B3
:102EB40074063EF583E5822DF582E5833CF583E0D7
:102EC400FCA3E0FD7804FFAE04088006A2E0CE1364
:102ED400CE13D8F8022F7EE55564016003022F87D4
:102EE400AF57EF3395E0FEEF25E0FDEE33FCAF5630
:102EF400EF3395E0FEEF7805C333CE33CED8F92413
:102F0400F0F58274103EF583E5822DF582E5833C6D
:102F1400F583E0FAA3E0FB780CFFAE02088006A27A
:102F2400E0CE13CE13D8F8540FF5587808AF03AE9B
:102F340002EF088006A2E0CE13CE13D8F8540FF5A2
:102F440059AF56EF3395E0FEEF7805C333CE33CE59
:102F5400D8F924F0F58274103EF583E5822DF582CC
:102F6400E5833CF583E0FCA3E0FD7804FFAE0408B0
:102F74008006A2E0CE13CE13D8F8540FF55AED54C0
:102F84000FF55BE558700FE559700BE55A7007E5CE
:102F94005B7003023019AD58E4FF127417AD59E4A5
:102FA400FF127417E55864097048855A5CAF5CFEDB
:102FB4007804EF08800633CE33CE92E0D8F8F55C7F
:102FC400E55B425CE55CB4990B7D09E4FF12741780
:102FD4007D098027E55C75F00A84F55DFDE4FF1248
:102FE4007417E55D75F00AA4FFC3E55C9FF55DFD0C
:102FF4008009AD5AE4FF127417AD5BE4FF12741735
:103004007FF47E011277B60557C3E557648094A018
:053014005003022E37FD
:013019002294
:0259D1008B51F8
:1059D30012646E8F52E552D394005003025A6DE560
:1059E3005294334003025A6DD269AF511257C27DAC
:1059F300527F05127417AF52124906744F2552F5A0
:105A030082E43406F583E060047D3880027D367FCE
:105A1300061274177F2C7E011277B67F2C7E01123B
:105A230077B675F020E552A424D0F582E5F034066C
:105A3300F583E0FEA3E0FF900000EEF0A3EFF04E4D
:105A430070077D1B7F061274177D0C7F031274177A
:105A5300900000E07002A3E06009E55214FDE4FF4A
:105A6300122E30C269AF510257C2C268AF511278C9
:015A7300EB47
:015A7400220F
:02623A008B5186
:10623C0012646EAD07EDD39400406BED9433506651
:10624C00E4FCECFF3395E0FEEF25E0FFEE33FE754A
:10625C00F020EDA424D0F582E5F03410F583E5822E
:10626C002FF582E5833EF583E4F0A3F00CBC10D24D
:10627C00749F2DF582E43406F583E4F0FCECFF33D7
:10628C0095E0FE75F008EDA424F8F582E5F03400F5
:10629C00F583E5822FF582E5833EF583E4F00CBCB3
:0D62AC0008DBD2688002C268AF511278EBA7
:0162B90022C2
:026825008B5195
:1068270012646EAD07EDD394004045ED94335040AC
:10683700E4FCECFF3395E0FEEF25E0FFEE33FE7559
:10684700F020EDA424D0F582E5F03406F583E58247
:106857002FF582E5833EF583E4F0A3F00CBC10D25C
:10686700744F2DF582E43406F583E4F0D268800294
:07687700C268AF511278EB7B
:01687E0022F7
:107244002430F58274003EF583EDF0AF55EF3395AD
:10725400E0FEE5522FF582E5513EF583A3A3E0FF5E
:10726400D3EF648094814008EF6480948A500122B3
:037274007F002276
:10788200D3EF648094804008EF648094A150012279
:037892007F002252
:081348008E518F528D538B541E
:101350008F828E83A3A3A3E014F55674FC2554F565
:10136000546403600FE55464076009E554640B603E
:10137000030216EBC3E5566480948050030216EB1B
:10138000E5566480948840030216EBE4F555AF56A9
:10139000EF3395E0FEEF7803C333CE33CED8F92494
:1013A00030F58274003EF583AF55EF3395E0FEE5EE
:1013B000822FF582E5833EF583E4F00555E555B4CB
:1013C00008CC755504E5546403705FAF55EF339551
:1013D000E0FEE5522FF582E5513EF583E0FFE5554D
:1013E000FD3395E0FCE5522DF582E5513CF583A3F4
:1013F000E0FD12646E127882AD07AF56EF3395E0D0
:10140000FEEF7803C333CE33CED8F9127244AD0762
:10141000AF56EF3395E0FEEF7803C333CE33CED82B
:10142000F92431F58274000216E2E5546407600382
:1014300002151DAF55EF3395E0FEE5522FF582E51D
:10144000513EF583E0FFE555FD3395E0FCE5522D77
:10145000F582E5513CF583A3E0FD12646E127882BB
:10146000AD07AF56EF3395E0FEEF7803C333CE33CD
:10147000CED8F9127244AD07AF56EF3395E0FEEFC8
:101480007803C333CE33CED8F92431F58274003ECD
:10149000F583EDF0AF55EF3395E0FEE5522FF58281
:1014A000E5513EF583A3127260AD07AF56EF339559
:1014B000E0FEEF7803C333CE33CED8F9126427129F
:1014C0007882AD07AF56EF3395E0FEEF7803C33374
:1014D000CE33CED8F92433F58274003EF583EDF097
:1014E000AF55EF3395E0FEE5522FF582E5513EF51D
:1014F00083E5822406F582E43583F583E0FF1272EA
:1015000064AD07AF56EF3395E0FEEF7803C333CEFB
:1015100033CED8F92434F58274000216E2E554641F
:101520000B60030216EBAF55EF3395E0FEE5522F4B
:10153000F582E5513EF583E0FFE555FD3395E0FC8E
:10154000E5522DF582E5513CF583A3E0FD12646E72
:10155000127882AD07AF56EF3395E0FEEF7803C304
:1015600033CE33CED8F9127244AD07AF56EF339570
:10157000E0FEEF7803C333CE33CED8F92431F582C1
:1015800074003EF583EDF0AF55EF3395E0FEE55284
:101590002FF582E5513EF583A3127260AD07AF5679
:1015A000EF3395E0FEEF7803C333CE33CED8F91294
:1015B0006427127882AD07AF56EF3395E0FEEF78DF
:1015C00003C333CE33CED8F92433F58274003EF50D
:1015D00083EDF0AF55EF3395E0FEE5522FF582E550
:1015E000513EF583E5822406F582E43583F583E0F8
:1015F000FF127264AD07AF56EF3395E0FEEF78034C
:10160000C333CE33CED8F92434F58274003EF5834B
:10161000EDF0AF55EF3395E0FEE5522FF582E55141
:101620003EF583E5822407F582E43583F583E0FF08
:10163000127264AD07AF56EF3395E0FEEF7803C347
:1016400033CE33CED8F92435F58274003EF583EDE0
:10165000F0AF55EF3395E0FEE5522FF582E5513EB0
:10166000F583E5822408F582E43583F583E0FFE520
:1016700055FD3395E0FCE5522DF582E5513CF583AF
:10168000E5822409126465127882AD07AF56EF3304
:1016900095E0FEEF7803C333CE33CED8F92436F588
:1016A0008274003EF583EDF0AF55EF3395E0FEE533
:1016B000522FF582E5513EF583E582240AF582E456
:1016C0003583F583E0FF127264AD07AF56EF3395B3
:1016D000E0FEEF7803C333CE33CED8F92437F5825A
:1016E00074003EF583EDF0D2688002C268AF5312F9
:0216F00078EB95
:0116F20022D5
:106D5200EF24FE601014601314601624037016D220
:106D620008D2248010D209D225800AD20ED22680DF
:106D720004D20CD2277FF47E011277B6753D04E56A
:106D82003D70FC7F647E001277B6C224C225C22603
:0B6D9200C227C208C209C20EC20C22B8
:107277008D51C3EF648094814026EF6480948A50D7
:107287001F126F09D267AF51125876753D017F32D1
:107297007E001277B6E53D70FCC267AF5112587693
:0172A70022C4
:046C1D008D51AC07E2
:106C2100D3EC64809480403CEC648094895035E4DA
:106C3100FDECFF3395E0FEEF7803C333CE33CED8BE
:106C4100F92428F58274003EF583EDFF3395E0FECB
:106C5100E5822FF582E5833EF583E4F00DBD08D191
:0B6C6100D2688002C268AF511278EBCD
:016C6C002205
:0442C1008C528D533B
:1042C500D3EF6480948050030243C9EF64809495D2
:1042D50040030243C9EB6480948750030243C9EB52
:1042E500648094E440030243C9EF3395E0FEEF7820
:1042F50005C333CE33CED8F92460F58274033EAFBF
:1043050082F5568F57EB24FBF558D39402500302E0
:1043150043C9E55875F00384E5F060030243C9E538
:104325005875F00384F55AC3941040030243C90538
:1043350057E557AE567002055614F5828E83E55A39
:10434500F074052553F553E43552F552E4F558E577
:1043550058C3955A506A855382855283E0F559B4FE
:104365000A130557E557AE567002055614F5828EA9
:1043750083E4F080120557E557AE567002055614D2
:10438500F5828E83E559F0855382855283A3E0FF3C
:10439500855382855283A3A3E0FD12774F8F59057C
:1043A50057E557AE567002055614F5828E83E559CA
:1043B500F074032553F553E43552F5520558808FB3
:0B43C500D2688002C268AF551278EB8E
:0143D00022CA
:0454D8008F518D5211
:1054DC00E551D39400500302558FE55194154003C8
:1054EC0002558FD269AF521257C27D5F7F0512747D
:1054FC0017AD51E4FF1274177D527F041274177F9D
:10550C00F47E011277B675F020E551A42460F58283
:10551C00E5F03403AF82F5558F56F583E0F5536013
:10552C004DD394004056E55394105050E55325E06C
:10553C00F553755401E5532401FFE433FEC3E554E0
:10554C009FEE6480F87480985032E5562554F582AD
:10555C00E43555F583E0FFE5562554F582E43555E1
:10556C00F583A3E0FD1274170554055480C77D1B09
:10557C007F061274177D5F7F05127417C269AF52D4
:0A558C000257C2C268AF521278EB5A
:0155960022F2
:1074BC008D51EFD3940A4006EFD3940F4003EF7035
:1074CC000E90063FEFF0D268AF511278EBD322C288
:0874DC0068AF511278EBC322E6
:1074E4008D51EFD3940A4006EFD3940F4003EF700D
:1074F4000E90063BEFF0D268AF511278EBD322C264
:0875040068AF511278EBC322BD
:106F4F008F52E552B40B067D5F7F078034E552B454
:106F5F000C067D5E7F068029E552B40D067D0A7F03
:106F6F0002801EE552B40E067D327F028013E55279
:106F7F00B40F067D467F028008E55270077D0A7FB9
:056F8F0003127417223B
:1073BF008F51D2691257C27D207F051274177D2E0F
:1073CF007F031274177D527F0412741790063FE0EB
:0C73DF00FF126F4FC269AF511257C2225B
:1073EB008F51D2691257C27D207F051274177D21F0
:1073FB007F061274177D527F0412741790063BE0C0
:0C740B00FF126F4FC269AF511257C2222E
:107655008D51D3EF64809480400EEF648094865002
:10766500071271A8D2688002C268AF511278EB2266
:0670CC008D51AB07AA067E
:1070D2008B828A83A3A3A3E0FFEB2404F582E43A24
:1070E20012646AD3EF648094804010EF648094A1AC
:1070F200500990063DEFF0D2688002C268AF51128B
:0271020078EB28
:017104002268
:0672D9008D51AB07AA066F
:1072DF008B828A83A3A3A3E0FFEB2404F582E43A15
:1072EF0012646AEFC39421500990063CEFF0D26804
:0972FF008002C268AF511278EB65
:017308002262
:065BB8008E518F528B5349
:105BBE00755406755540D3ED64809484407CED6435
:105BCE008094A55075ED24FDF556D39404406BE5F5
:105BDE005620E06613F5570555E555AE547002058F
:105BEE005414F5828E83E557F074032552F552E472
:105BFE003551F551E4F556E556C395575033855258
:105C0E0082855183E0FFA3E0FD12774F0555E555E0
:105C1E00AC547002055414F5828C83EFF00552E5F6
:105C2E0052700205510552E552700205510556801B
:105C3E00C6D268AF531278EBD322C268AF53127834
:025C4E00EBC3A6
:015C50002231
:0843D1008E518F528D538B5465
:1043D900C267D3E553648094845003024486E5534D
:1043E9006480948D40030244868F828E83A3A3E068
:1043F900640A60030244868F828E83A3A3A3E01418
:10440900B40800507690441C75F003A4C58325F0C8
:10441900C5837302443402443E02444802445202B2
:10442900445C02446602447002447A75550075562C
:1044390080D2678048755500755688D267803E7569
:104449005500755690D2678034755500755698D2C7
:1044590067802A7555007556A0D26780207555006A
:104469007556A8D26780167555007556B0D2678003
:104479000C755500755678D2678002C2673067504F
:10448900E4FFEF7C002556FDEC35558D82F583E47C
:10449900F00FBF08EDE55324FB855682855583F05F
:1044A9007F01E5522404F582E43551F583E5822F35
:1044B900F582E43583F583E0FEEF7C002556FDECBB
:1044C90035558D82F583EEF00FBF08D6D26880028C
:0744D900C268AF541278EB3A
:0144E00022B9
:045EA0008E548F5538
:105EA4000555E5557002055414F5828E83E0F557C7
:105EB4006074C39408506F7F2C7E011277B6E4F5AA
:105EC40056E556C39557505E855582855483E060E8
:105ED4003624F5601414601714601A14601D1460DD
:105EE4002024057028E4FD802D7D5F7F0780287DB8
:105EF4005E7F0680227D0A7F02801C7D327F0280C5
:105F0400167D467F0280107D0A7F03800A855582B4
:105F1400855483E0FDE4FF1274170555E5557002BE
:065F240005540556809BA8
:015F2A002254
:022C3C008B51BA
:102C3E00C267EF640A6003022E17ED14B408004059
:102C4E0003022E15902C6075F003A4C58325F0C5E4
:102C5E008373022C78022CAC022CE0022D14022D70
:102C6E0048022D7C022DAF022DE2D269AF511257D0
:102C7E00C27D577F021274177D05E4FF127417E4AC
:102C8E00FDFF1274177D01E4FF1274177D527F044D
:102C9E00127417755200755380D267022E17D269BF
:102CAE00AF511257C27D577F021274177D05E4FF94
:102CBE00127417E4FDFF1274177D02E4FF127417ED
:102CCE007D527F04127417755200755388D26702B5
:102CDE002E17D269AF511257C27D577F0212741749
:102CEE007D05E4FF127417E4FDFF1274177D03E4F3
:102CFE00FF1274177D527F041274177552007553AC
:102D0E0090D267022E17D269AF511257C27D577FEC
:102D1E00021274177D05E4FF127417E4FDFF12749E
:102D2E00177D04E4FF1274177D527F041274177519
:102D3E005200755398D267022E17D269AF511257AF
:102D4E00C27D577F021274177D05E4FF127417E4DB
:102D5E00FDFF1274177D05E4FF1274177D527F0478
:102D6E001274177552007553A0D267022E17D269CE
:102D7E00AF511257C27D577F021274177D05E4FFC3
:102D8E00127417E4FDFF1274177D06E4FF12741718
:102D9E007D527F041274177552007553A8D2678046
:102DAE0068D269AF511257C27D577F021274177DD8
:102DBE0005E4FF127417E4FDFF1274177D07E4FF9C
:102DCE001274177D527F041274177552007553B02A
:102DDE00D2678035D269AF511257C27D577F02122A
:102DEE0074177D05E4FF127417E4FDFF1274177D4E
:102DFE0008E4FF1274177D527F0412741775520087
:102E0E00755378D2678002C267306709AF53AE52EE
:102E1E00125EA08005AF51127761C269AF51125791
:012E2E00C2E1
:012E2F002280
:08301A008E518F528D538B542F
:10302200C2678F828E83A3A3E0640A60030230D159
:103032001247FF8E568F57D3E557943BE5569400BF
:1030420050030230CCE5579408E5569407507BC3F1
:10305200E5536480948A5072855282855183A3A37A
:10306200A3E0F555B40106900600023177E555B4A8
:103072000206900602023177E555B4030690060473
:10308200023177E555B40406900606023177E5551C
:10309200B40506900608023177E555B40606900697
:1030A2000A023177E555B4070690060C023177E53E
:1030B20055B4080690060E023177E555B40906901C
:1030C2000610023177D2670231F3D2670231F385FB
:1030D2005282855183A3A3E064016003023181AD72
:1030E20053AF52AE511247FF8E568F57D3E55794C6
:1030F2003BE556940050030231F3E5579408E55638
:10310200940740030231F3C3E5536480948A400379
:103112000231F3855282855183A3A3A3E0F555B40E
:103122000A05900612804EE555B4010590061480FA
:1031320044E555B40205900616803AE555B40305F8
:103142009006188030E555B4040590061A8026E5ED
:1031520055B4050590061C801CE555B4060590067D
:103162001E8012E555B407059006208008E555B487
:103172000809900622E556F0A3806FD26780728517
:103182005282855183A3A3E064027065AD53AF52AE
:10319200AE5112687F7556008F57C3E5579463E5A9
:1031A200569400504CC3E553648094885043855232
:1031B20082855183A3A3A3E0F555B401079006309D
:1031C200EFF0802DE555B40205900631801CE555DF
:1031D200B403059006328012E555B4040590063317
:1031E2008008E555B40508900634E557F08002D210
:0F31F20067306704C2688002D268AF541278EB6E
:0132010022AA
:102539008F518D528B53E551640A60030225E5E5FD
:1025490052C3940A40030227BBD269AF531257C240
:102559007D277F081274177D06E4FF127417E4FDC6
:10256900FF127417AD52E4FF1274177D527F0412E3
:102579007417E55214B4090040030227B490259456
:1025890075F003A4C58325F0C583730225AF022521
:10259900B50225BB0225C10225C70225CD0225D3D7
:1025A9000225D90225DF9006000226F590060202CF
:1025B90026F59006040226F59006060226F59006F1
:1025C900080226F590060A0226F590060C0226F561
:1025D90090060E0226F59006100226F5E5516401D3
:1025E9006003022703E552D394004006E55294099B
:1025F9004009E552640A6003022700D269AF531209
:1026090057C27D277F081274177D06E4FF127417DD
:10261900E552B40A147D0AE4FF1274177D527F044F
:102629001274179006120226F5E552B401147D0BB7
:10263900E4FF1274177D527F041274179006140276
:1026490026F5E552B402147D0CE4FF1274177D528D
:102659007F041274179006160226F5E552B4031387
:102669007D0DE4FF1274177D527F041274179006D2
:10267900188079E552B404137D0EE4FF1274177DB6
:10268900527F0412741790061A8061E552B405133B
:102699007D0FE4FF1274177D527F041274179006A0
:1026A9001C8049E552B406137D10E4FF1274177DAE
:1026B900527F0412741790061E8031E552B4071335
:1026C9007D11E4FF1274177D527F0412741790066E
:1026D900208019E552640860030227C27D12FF12A7
:1026E90074177D527F04127417900622E0FEA3E04E
:1026F900FF1272A80227C20227BBE55164026003D8
:102709000227C2E552D3940050030227BBE5529435
:102719000740030227BBD269AF531257C27D277FF7
:10272900081274177D06E4FF1274177D14E4FF1272
:102739007417E55224FE6020146030146040146060
:1027490050240470667D01E4FF1274177D527F04E2
:10275900127417900630804A7D02E4FF1274177DC7
:10276900527F0412741790063180377D03E4FF12FB
:1027790074177D527F0412741790063280247D04E9
:10278900E4FF1274177D527F041274179006338088
:10279900117D05E4FF1274177D527F04127417909E
:1027A9000634E0FF7E00127309800EAF5312776181
:1027B9008007C268AF531278EBC269AF531257C290
:0127C90022ED
:0647FF008E588F59A90538
:104805007D057C00E5592DF582E5583CF583E0C32F
:10481500940A400CE5592DF582E5583CF583E4F002
:104825000DBD00010CED640A4C70D9B90610E559AF
:104835002405F582E43558F583E0FF7E0022E9641E
:10484500077019E5592405F582E43558F583E075B7
:10485500F00AA4ACF0FDE55924068032E96408703D
:104865003DE5592405F582E43558F583E075F06496
:10487500A4ACF0FDE5592406F582E43558F583E04E
:1048850075F00AA42DFDE5F03CFCE5592407F582F9
:10489500E43558F583E02DFDE43CAF05FE22E964DF
:1048A50009705AE5592405F582E43558F583E0FF8A
:1048B5007E007C037DE8125675AC06AD07E55924EC
:1048C50006F582E43558F583E075F064A42DFDE521
:1048D500F03CFCE5592407F582E43558F583E0758D
:1048E500F00AA42DFDE5F03CFCE5592408F582E429
:1048F5003558F583E02DFDE43CFEAF0522E4FEFFCF
:01490500228F
:06687F008E588F59A90597
:106885007F057E00E5592FF582E5583EF583E0C387
:10689500940A400CE5592FF582E5583EF583E4F05E
:1068A5000FBF00010EEF64084E70D9E96407702030
:1068B500E5592405F582E43558F583E075F00AA419
:1068C500FFE5592406F582E43558F583E02FFF22CC
:0268D5007F0042
:0168D700229E
:104906008F56E556D3945940147D5AE4FF12741716
:10491600E55624A6FD7003024A07024A02E556D36D
:10492600944F401AE556945A50147D50E4FF127481
:1049360017E55624B0FD7003024A07024A02E556FF
:10494600D39445401AE556945050147D46E4FF1220
:104956007417E55624BAFD7003024A07024A02E5B7
:1049660056D3943B4019E556944650137D3CE4FFDC
:10497600127417E55624C4FD7003024A07807DE5CC
:1049860056D394314016E556943C50107D32E4FFE0
:10499600127417E55624CEFD60678060E556D39401
:1049A600274016E556943250107D28E4FF127417FE
:1049B600E55624D8FD604A8043E556D3941D40163B
:1049C600E556942850107D1EE4FF127417E5562410
:1049D600E2FD602D8026E556D394134016E55694E5
:1049E6001E50107D14E4FF127417E55624ECFD608A
:1049F600108009E556C394145007AD56E4FF1274AF
:024A0600172275
:107309008E548F557C007D0A125687AD07E4FF1213
:1073190074177D5B7F06127417AE54AF557C007DE0
:107329000A125687E4FF1274177D4A7F0702741701
:0472A8008E548F551C
:1072AC007C007D3C1256871249067D057F061274C0
:1072BC0017AE54AF557C007D3C125687ED4C600CDC
:0C72CC00AF051249067D4A7F07127417B7
:0172D8002293
:026DE7008D51CC
:106DE900D3EF648094804038EF648094955031EFFC
:106DF9003395E0FEEF7805C333CE33CED8F924605E
:106E0900F58274033EAF82FEE4FD0FEFAA0670011E
:106E19000E14F5828A83E4F00DBD20EED26880025B
:076E2900C268AF511278EBC3
:016E3000223F
:107053008F51900640E0D394024015D267125876C0
:10706300753D037F327E001277B6E53D70FC8015D7
:10707300D267AF511258767D1B7F061274177D0CB1
:0D7083007F03127417C267AF5112587622B6
:1078B9007E10900640E4F0A3DEFC7E10D2681278B8
:0178C900EBD3
:0178CA00229B
:1075EF008F5CD2691257C27D607F021274177D3291
:1075FF007F061274177D1E7F05127417C269AF5C68
:04760F001257C2222A
:107761008F5CD2691257C27D607F021274177D301F
:0D7771007F03127417C269AF5C1257C22269
:0E78EB008F5B3068030275EFAF5B127761228E
:106427002432F58274003EF583EDF0AF55EF3395D6
:10643700E0FEE5522FF582E5513EF583E58224041F
:10644700F582E43583F583E0FFE555FD3395E0FC00
:10645700E5522DF582E5513CF583E5822405F58269
:07646700E43583F583E0FD3D
:10646E00EFD394004015EF940B5010EFC3940A50E5
:10647E0008EF75F00AA4FE8002E4FEEDD39400400E
:10648E000EED940B5009EDC3940A5003ED2EFEAFA2
:01649E0006F7
:01649F0022DA
:030000000278DCA7
:0F78DC00758E0078FEE4F6D8FD75816C024FD1F1
:10780500D292C0F075F008C29100A29233D291D500
:06781500F0F5D0F0FF22A7
:10781B00EFC0F075F00833C291929333D291D5F04B
:06782B00F6D0F0C291222C
:10741700EFFEEDFF1280008E2F8F30125A75755FC9
:1074270064AF5F155FEFD39400400EE4F55EE55E51
:09743700C3943A50EC055E80F5A7
:017440002229
:105A7500D2A885A86175A881C244853082852F8307
:105A8500E493F560C4540FF5604360F0856080C20F
:105A950084D28500C2870000D287007580FF75809B
:105AA500FEC284C28500C28700000000D28700754F
:105AB50080FFD24475623E756380E4F56030941DC5
:105AC5000560E560B464F6123202E56315637002A1
:105AD5001562D3E5639400E562940050DD75623E7E
:105AE500756380E4F56020941D0560E560B464F697
:105AF500123202E563156370021562D3E563940003
:105B0500E562940050DD8561A8C2A87F147E00126D
:025B150077B661
:015B1700226B
:107441007580FDC284C28500C28700000000D2871A
:10745100007580FF7F147E001277B67F997E091236
:0A74610080008E2F8F30125A752222
:10565300C2D530F707B2D563F0FF05F030E70CB2DF
:10566300D5F4048463F0FF05F080018430D502F49F
:0256730004220F
:10567500EF8DF0A4A8F0CF8CF0A428CE8DF0A42E49
:02568500FE2203
:10568700BC000BBE0029EF8DF084FFADF022E4CC07
:10569700F875F008EF2FFFEE33FEEC33FCEE9DECD0
:1056A700984005FCEE9DFE0FD5F0E9E4CEFD22ED16
:1056B700F8F5F0EE8420D21CFEADF075F008EF2F60
:1056C700FFED33FD4007985006D5F0F222C398FD51
:0556D7000FD5F0EA22EE
:1056DC00EB9FF5F0EA9E42F0E99D42F0E89C45F024
:0156EC00229B
:1056ED007401FF3395E0FEFDFC080808E6CF2FF6A8
:1056FD0018E6CE3EF618E6CD3DF618E6CC3CF62281
:1078CB00EFC39461400AEF947B5005EF24E0FF2255
:0178DB00228A
:00000001FF
